:100000000C944D010C946A010C946A010C946A01E1
:100010000C946A010C946A010C946A010C946A01B4
:100020000C946A010C946A010C946A010C946A01A4
:100030000C946A010C9481110C94B4110C94A210CC
:100040000C944E110C94E8100C941B110C946A0142
:100050000C946F100C946A010C946A010C941610A5
:100060000C946A010C945C0B0C946A010C94B00A19
:100070000C946A010C94A4020C946A010C946A0119
:100080000C946A010C946A010C946A010C946A0144
:100090000C94870B0C946A010C94DB0A0C946A0193
:1000A0000C946A010C946A010C946A010C946A0124
:1000B0000C946A010C946A010C946A010C946A0114
:1000C0000C946A010C946A010C946A010C94B20BB2
:1000D0000C946A010C94060B0C94DD0B0C946A01D1
:1000E0000C94310B000001000800400000010004E6
:1000F0000000010008002000400080000001000412
:10010000303132333435363738394142434445464D
:10011000000D0A0D0A002563006100593D25642089
:10012000553D256420563D25640D0A0D0A00766D67
:1001300000523D256420473D256420423D25640D45
:100140000A0D0A002564256425640D0A002564252E
:1001500064256400256425642564002564256425E0
:1001600064002564256425640025642564256400F5
:100170007663256400256425642564002564256470
:1001800025640025642564256400256425642564B0
:1001900000256425642564002564256425640076B3
:1001A000632564002C20583D256420593D25640DAD
:1001B0000A0D0A00585F6C6566743D25642C205852
:1001C0005F72696768743D256420595F746F703D84
:1001D000256420595F626F74746F6D3D25642050F3
:1001E00069783D2564007662256400203300203262
:1001F0000020310020300020330020320020310068
:10020000203000203300203200203000383A2564AE
:1002100020393A25642031303A25642031313A259D
:10022000642031323A25642031333A256420313458
:100230003A25642031353A2564200D0A00303A25EC
:100240006420313A256420323A256420333A25640B
:1002500020343A256420353A256420363A25642036
:10026000373A2564200D0A00496E697469616C692A
:100270007A6174696F6E20436F6D706C6574652070
:100280000D0A002E000D0A53797374656D205761B5
:10029000726D696E67205570000011241FBECFEF8C
:1002A000D1E2DEBFCDBF12E0A0E0B2E0EEE1F1E6C8
:1002B00002C005900D92A23CB107D9F716E0A2EC5E
:1002C000B2E001C01D92A130B107E1F70E94142EE7
:1002D0000C948E300C940000CF93DF93CDB7DEB733
:1002E000AAE7B0E0EAE7F0E0808180688C93AAE7B3
:1002F000B0E0EAE7F0E080818F7D8C9386E00E9499
:10030000AE0181E00E94CC01ACE7B0E0ECE7F0E0A8
:1003100080818F7D8C93AAE7B0E0EAE7F0E08081EE
:1003200088608C9310921A057894DF91CF9108958C
:10033000CF93DF93CDB7DEB7AAE7B0E0EAE7F0E00E
:100340008081877F8C93AAE7B0E0EAE7F0E09081B4
:100350008FE789238C93DF91CF910895CF93DF931B
:10036000CDB7DEB721970FB6F894DEBF0FBECDBF75
:100370008983AAE7B0E0EAE7F0E08081982F987FD0
:100380008981892B8C9321960FB6F894DEBF0FBE1E
:10039000CDBFDF91CF910895CF93DF93CDB7DEB777
:1003A00021970FB6F894DEBF0FBECDBF8983ACE7AF
:1003B000B0E0ECE7F0E08081982F8FE3292F28232D
:1003C0008981882F90E000249695879507949695CB
:1003D00087950794982F802D822B8C9321960FB6AA
:1003E000F894DEBF0FBECDBFDF91CF910895CF93BC
:1003F000DF93CDB7DEB721970FB6F894DEBF0FBEFF
:10040000CDBF8983ACE7B0E0ECE7F0E08081982FC6
:10041000907E89818F71892B8C9321960FB6F894E9
:10042000DEBF0FBECDBFDF91CF910895CF93DF9395
:10043000CDB7DEB7AAE7B0E0EAE7F0E080818061FF
:100440008C93AAE7B0E0EAE7F0E0808180648C93C7
:10045000DF91CF910895CF93DF93CDB7DEB7EAE771
:10046000F0E08081882F90E080749070DF91CF91D0
:100470000895CF93DF93CDB7DEB721970FB6F894E9
:10048000DEBF0FBECDBF898310921A0589818830E7
:1004900040F0ABE7B0E0EBE7F0E0808188608C9360
:1004A00007C0ABE7B0E0EBE7F0E08081877F8C939B
:1004B000ACE7B0E0ECE7F0E08081982F987F89818D
:1004C0008770892B8C93AAE7B0E0EAE7F0E080819F
:1004D00080618C93AAE7B0E0EAE7F0E08081806475
:1004E0008C93EAE7F0E08081882F90E08074907030
:1004F0000097B9F7E8E7F0E08081918121960FB687
:10050000F894DEBF0FBECDBFDF91CF910895CF939A
:10051000DF93CDB7DEB721970FB6F894DEBF0FBEDD
:10052000CDBF898389810E943902969587959695DA
:100530008795882F90E021960FB6F894DEBF0FBE06
:10054000CDBFDF91CF9108951F920F920FB60F92FA
:1005500011248F93CF93DF93CDB7DEB78FEF8093C6
:100560001A05DF91CF918F910F900FBE0F901F90C2
:100570001895CF93DF93CDB7DEB727970FB6F894D2
:10058000DEBF0FBECDBF9B838A837D836C835F8379
:100590004E83EFE5F0E080818983F894EA81FB8166
:1005A0008C819D8191838083EA81FB818E819F81F3
:1005B00093838283EA81FB8117821682EA81FB8121
:1005C00015821482EFE5F0E08981808327960FB6CB
:1005D000F894DEBF0FBECDBFDF91CF910895CF93CA
:1005E000DF93CDB7DEB724970FB6F894DEBF0FBE0A
:1005F000CDBF9C838B831A82EFE5F0E080818983F5
:10060000F894EB81FC81848195810097D1F1EB8195
:10061000FC8120813181EB81FC8186819781F90108
:10062000E80FF91F80818A83EB81FC8186819781A5
:100630000196EB81FC8197838683EB81FC81268187
:100640003781EB81FC81828193812817390780F003
:10065000EB81FC8126813781EB81FC818281938152
:10066000A901481B590BCA01EB81FC819783868342
:10067000EB81FC81848195810197EB81FC819583DD
:100680008483EFE5F0E0898180838A81882F90E080
:1006900024960FB6F894DEBF0FBECDBFDF91CF9189
:1006A0000895CF93DF93CDB7DEB725970FB6F894B3
:1006B000DEBF0FBECDBF9B838A837D836C83EFE556
:1006C000F0E080818983F894EA81FB81248135817F
:1006D0008C819D8182179307B0F5EA81FB81268189
:1006E00037818C819D81820F931FEA81FB819783E3
:1006F0008683EA81FB8126813781EA81FB818281C1
:1007000093812817390780F0EA81FB8126813781A0
:10071000EA81FB8182819381A901481B590BCA019F
:10072000EA81FB8197838683EA81FB81248135817D
:100730008C819D81A901481B590BCA01EA81FB816B
:100740009583848304C0EA81FB8115821482EFE5DE
:10075000F0E08981808325960FB6F894DEBF0FBE46
:10076000CDBFDF91CF9108950F931F93CF93DF9368
:10077000CDB7DEB726970FB6F894DEBF0FBECDBF5C
:100780009C838B837E836D83EFE5F0E080818A8399
:10079000F894EB81FC8100811181EB81FC81268141
:1007A00037818D819E81820F931FEB81FC81228195
:1007B0003381B9010E942A30F801E80FF91F8081C6
:1007C0008983EFE5F0E08A8180838981882F90E03A
:1007D00026960FB6F894DEBF0FBECDBFDF91CF9146
:1007E0001F910F9108950F931F93CF93DF93CDB770
:1007F000DEB726970FB6F894DEBF0FBECDBF9B8342
:100800008A836C83EFE5F0E080818983F894EA8144
:10081000FB8124813581EA81FB81828193812817C4
:10082000390760F5EA81FB8100811181EA81FB8152
:1008300026813781EA81FB8184819581820F931F14
:10084000EA81FB8122813381B9010E942A30F801BB
:10085000E80FF91F8C818083EA81FB818481958177
:100860000196EA81FB8195838483EFE5F0E089813D
:1008700080838FEF90E09E838D8306C0EFE5F0E0EC
:10088000898180831E821D828D819E8126960FB66E
:10089000F894DEBF0FBECDBFDF91CF911F910F91B6
:1008A0000895CF93DF93CDB7DEB725970FB6F894B1
:1008B000DEBF0FBECDBF9D838C83EFE5F0E080816E
:1008C0008B83F894EC81FD8122813381EC81FD8161
:1008D00084819581A901481B590BCA019A83898398
:1008E000EFE5F0E08B81808389819A8125960FB6B0
:1008F000F894DEBF0FBECDBFDF91CF910895CF93A7
:10090000DF93CDB7DEB723970FB6F894DEBF0FBEE7
:10091000CDBF9B838A83EFE5F0E080818983F894E3
:10092000EA81FB8115821482EFE5F0E08981808302
:1009300023960FB6F894DEBF0FBECDBFDF91CF91E7
:100940000895CF93DF93CDB7DEB70E94B0040E9425
:10095000D2040E94F4040E941605DF91CF910895FD
:10096000CF93DF93CDB7DEB70E9438051092030511
:1009700010920205E1ECF0E088ED808340E855E25A
:1009800060E070E080E00E94C9058FEF80931B0556
:1009900010923F0510926405109263057894DF91E0
:1009A000CF910895CF93DF93CDB7DEB70E94530563
:1009B0001092050510920405E9ECF0E088ED8083C3
:1009C00040E855E260E070E081E00E94C9058FEFE9
:1009D00080931C05109240051092660510926505E3
:1009E0007894DF91CF910895CF93DF93CDB7DEB7A1
:1009F0000E946E051092070510920605E1EDF0E0E9
:100A000088ED808340E855E260E070E082E00E947B
:100A1000C9058FEF80931D0510924105109268055E
:100A2000109267057894DF91CF910895CF93DF936B
:100A3000CDB7DEB70E94890510920905109208050E
:100A4000E1E3F1E088ED808340E855E260E070E0AA
:100A500083E00E94C9058FEF80931E051092420526
:100A600010926A05109269057894DF91CF910895EC
:100A7000CF93DF93CDB7DEB782EC92E02FE135E084
:100A800040E850E0BC01C9010E94B90282E493E051
:100A900023E435E040E150E0BC01C9010E94B90205
:100AA000DF91CF910895CF93DF93CDB7DEB782E585
:100AB00093E027E235E040E850E0BC01C9010E9424
:100AC000B90282ED93E02BE435E040E150E0BC0157
:100AD000C9010E94B902DF91CF910895CF93DF93AE
:100AE000CDB7DEB782EE93E02FE235E040E850E08C
:100AF000BC01C9010E94B90282E694E023E535E019
:100B000040E150E0BC01C9010E94B902DF91CF91E0
:100B10000895CF93DF93CDB7DEB782E794E027E364
:100B200035E040E850E0BC01C9010E94B90282EF03
:100B300094E02BE535E040E150E0BC01C9010E94A2
:100B4000B902DF91CF910895CF93DF93CDB7DEB790
:100B500023970FB6F894DEBF0FBECDBF89837B838A
:100B60006A838981843060F48981882F90E0880FBE
:100B7000991FFC01EE5FFA4F8A819B8191838083EC
:100B800023960FB6F894DEBF0FBECDBFDF91CF9195
:100B90000895EF92FF920F931F93CF93DF93CDB7FA
:100BA000DEB727970FB6F894DEBF0FBECDBF8B839D
:100BB0004C835D836E837F838C819D81AE81BF81F9
:100BC000880F991FAA1FBB1F880F991FAA1FBB1F41
:100BD000880F991FAA1FBB1F0F2EF0E0EF2EF4E223
:100BE000FF2EF4EF0F2FF0E01F2FF02DE80EF91E6F
:100BF0000A1F1B1F8C819D81AE81BF81880F991FA9
:100C0000AA1FBB1F880F991FAA1FBB1F880F991F00
:100C1000AA1FBB1F880F991FAA1FBB1F9C01AD01F4
:100C2000C801B7010E945130DA01C90101979A83C6
:100C300089838B81833061F4E4E3F1E089818083EF
:100C4000E5E3F1E089819A81892F9927808329C082
:100C50008B81823061F4E4EDF0E089818083E5ED01
:100C6000F0E089819A81892F992780831AC08B812E
:100C7000813061F4ECECF0E089818083EDECF0E010
:100C800089819A81892F992780830BC0E4ECF0E059
:100C900089818083E5ECF0E089819A81892F992709
:100CA000808327960FB6F894DEBF0FBECDBFDF91CD
:100CB000CF911F910F91FF90EF900895CF93DF9305
:100CC000CDB7DEB721970FB6F894DEBF0FBECDBF0C
:100CD00089838981882F90E0880F991F880F991F39
:100CE000880F991F815E9A4F21960FB6F894DEBF48
:100CF0000FBECDBFDF91CF910895CF93DF93CDB7D6
:100D0000DEB721970FB6F894DEBF0FBECDBF898343
:100D10008981882F90E0880F991F880F991F880F6D
:100D2000991F8D5B9A4F21960FB6F894DEBF0FBEC8
:100D3000CDBFDF91CF910895CF93DF93CDB7DEB7CD
:100D400022970FB6F894DEBF0FBECDBF89836A83AA
:100D50008981833071F4E0E3F1E08081882F90E0B5
:100D6000807290700097B9F3E6E3F1E08A818083A6
:100D70002FC08981823071F4E0EDF0E08081882F0E
:100D800090E0807290700097B9F3E6EDF0E08A8110
:100D900080831EC08981813071F4E8ECF0E08081AD
:100DA000882F90E0807290700097B9F3EEECF0E03D
:100DB0008A8180830DC0E0ECF0E08081882F90E094
:100DC000807290700097B9F3E6ECF0E08A8180833E
:100DD0008981882F90E0FC01E55EFA4F108222960F
:100DE0000FB6F894DEBF0FBECDBFDF91CF9108954F
:100DF000CF93DF93CDB7DEB721970FB6F894DEBF60
:100E00000FBECDBF8983698180E00E949C06219638
:100E10000FB6F894DEBF0FBECDBFDF91CF9108951E
:100E2000CF93DF93CDB7DEB721970FB6F894DEBF2F
:100E30000FBECDBF8983698181E00E949C06219607
:100E40000FB6F894DEBF0FBECDBFDF91CF910895EE
:100E5000CF93DF93CDB7DEB721970FB6F894DEBFFF
:100E60000FBECDBF8983698182E00E949C062196D6
:100E70000FB6F894DEBF0FBECDBFDF91CF910895BE
:100E8000CF93DF93CDB7DEB721970FB6F894DEBFCF
:100E90000FBECDBF8983698183E00E949C062196A5
:100EA0000FB6F894DEBF0FBECDBFDF91CF9108958E
:100EB000CF93DF93CDB7DEB723970FB6F894DEBF9D
:100EC0000FBECDBFCE010196BC0180E00E94F407A9
:100ED000882331F08981282F30E03B832A8304C0A6
:100EE0008FEF9FEF9B838A838A819B8123960FB626
:100EF000F894DEBF0FBECDBFDF91CF910895CF93A1
:100F0000DF93CDB7DEB723970FB6F894DEBF0FBEE1
:100F1000CDBFCE010196BC0181E00E94F407882379
:100F200031F08981282F30E03B832A8304C08FEF82
:100F30009FEF9B838A838A819B8123960FB6F894C7
:100F4000DEBF0FBECDBFDF91CF910895CF93DF936A
:100F5000CDB7DEB723970FB6F894DEBF0FBECDBF77
:100F6000CE010196BC0182E00E94F407882331F093
:100F70008981282F30E03B832A8304C08FEF9FEFC5
:100F80009B838A838A819B8123960FB6F894DEBF68
:100F90000FBECDBFDF91CF910895CF93DF93CDB733
:100FA000DEB723970FB6F894DEBF0FBECDBFCE01DC
:100FB0000196BC0183E00E94F407882331F0898107
:100FC000282F30E03B832A8304C08FEF9FEF9B8361
:100FD0008A838A819B8123960FB6F894DEBF0FBE69
:100FE000CDBFDF91CF910895CF93DF93CDB7DEB71B
:100FF00025970FB6F894DEBF0FBECDBF89837B83E4
:101000006A838981882F90E0880F991F880F991F24
:10101000880F991FFC01EF5DFA4F80819181009745
:1010200041F18981882F90E0880F991F880F991FBF
:10103000880F991FFC01ED5DFA4F80819181009727
:10104000A9F08981882F90E0880F991F880F991F38
:10105000880F991F815E9A4F0E94EF02EA81FB81FF
:1010600080838FEF90E09D838C8305C01D821C825E
:1010700002C01D821C828C819D8125960FB6F8943A
:10108000DEBF0FBECDBFDF91CF910895CF93DF9329
:10109000CDB7DEB721970FB6F894DEBF0FBECDBF38
:1010A00089838981882F90E0880F991F880F991F65
:1010B000880F991F815E9A4F0E947F0421960FB678
:1010C000F894DEBF0FBECDBFDF91CF910895CF93CF
:1010D000DF93CDB7DEB723970FB6F894DEBF0FBE10
:1010E000CDBF89838981882F90E0880F991F880F51
:1010F000991F880F991FFC01ED5DFA4F8081918146
:101100001B821A82009721F481E090E09B838A83FE
:101110008A819B8123960FB6F894DEBF0FBECDBFA8
:10112000DF91CF910895CF93DF93CDB7DEB72297AC
:101130000FB6F894DEBF0FBECDBF89836A83898165
:10114000882F90E0880F991F880F991F880F991F8B
:101150008D5B9A4F6A810E94F30322960FB6F89432
:10116000DEBF0FBECDBFDF91CF910895CF93DF9348
:10117000CDB7DEB721970FB6F894DEBF0FBECDBF57
:101180008983698180E00E94930821960FB6F894C4
:10119000DEBF0FBECDBFDF91CF910895CF93DF9318
:1011A000CDB7DEB721970FB6F894DEBF0FBECDBF27
:1011B0008983698181E00E94930821960FB6F89493
:1011C000DEBF0FBECDBFDF91CF910895CF93DF93E8
:1011D000CDB7DEB721970FB6F894DEBF0FBECDBFF7
:1011E0008983698182E00E94930821960FB6F89462
:1011F000DEBF0FBECDBFDF91CF910895CF93DF93B8
:10120000CDB7DEB721970FB6F894DEBF0FBECDBFC6
:101210008983698183E00E94930821960FB6F89430
:10122000DEBF0FBECDBFDF91CF910895CF93DF9387
:10123000CDB7DEB721970FB6F894DEBF0FBECDBF96
:1012400089838981882F90E0FC01E15CFA4F8FEF60
:1012500080838981882F90E0880F991F880F991FBC
:10126000880F991F8D5B9A4F0E94EF02682F89812A
:101270000E949C0621960FB6F894DEBF0FBECDBF2C
:10128000DF91CF910895CF93DF93CDB7DEB72A9743
:101290000FB6F894DEBF0FBECDBF89837B836A8310
:1012A0005D834C838981882F90E0880F991F880F78
:1012B000991F880F991FFC01E95BFA4F208131814A
:1012C0008C819D81280F391F8981882F90E0880F9C
:1012D000991F880F991F880F991FFC01EB5BFA4F2C
:1012E000808191812817390708F046C08C819D8143
:1012F000009709F441C0EA81FB81E081E8878A8197
:101300009B8101969B838A831F821E821CC0EA8177
:10131000FB8120818A819B8101969B838A838981BD
:10132000882F90E0880F991F880F991F880F991FA9
:101330008D5B9A4F622F0E94F3032E813F812F5FB6
:101340003F4F3F832E838C819D8101972E813F816A
:1013500028173907E0F28981882F90E0FC01E15CD1
:10136000FA4F8FEF8083688589810E949C068FEFFA
:1013700090E09A87898702C01A86198689859A859E
:101380002A960FB6F894DEBF0FBECDBFDF91CF9186
:1013900008950F931F93CF93DF93CDB7DEB72197B7
:1013A0000FB6F894DEBF0FBECDBF89838981882F29
:1013B00090E0FC01E15CFA4F8081882309F44DC084
:1013C0008981882F90E0880F991F880F991F880FB7
:1013D000991FFC01E95BFA4F80819181009769F1C7
:1013E0008981833049F406E311E08BE595E00E94A2
:1013F000EF02F801808339C08981823049F406ED1B
:1014000010E083E595E00E94EF02F80180832DC093
:101410008981813049F40EEC10E08BE495E00E9464
:10142000EF02F801808321C006EC10E083E495E030
:101430000E94EF02F801808318C08981882F90E014
:10144000FC01E15CFA4F10828981882F90E0FC0159
:10145000E55EFA4F8FEF808308C08981882F90E086
:10146000FC01E55EFA4F8FEF808321960FB6F8946A
:10147000DEBF0FBECDBFDF91CF911F910F910895B9
:10148000CF93DF93CDB7DEB722970FB6F894DEBFC8
:101490000FBECDBF8A838A81833029F4E6E3F1E071
:1014A0008081898314C08A81823029F4E6EDF0E0DE
:1014B000808189830CC08A81813029F4EEECF0E0D0
:1014C0008081898304C0E6ECF0E0808189838A8191
:1014D000882F90E0880F991FFC01EE5FFA4F808102
:1014E0009181009771F08A81882F90E0880F991F71
:1014F000FC01EE5FFA4F0190F081E02D8981199592
:1015000026C08A81882F90E0880F991F880F991F25
:10151000880F991F815E9A4F69810E94F303882387
:10152000B1F48A81282F30E0C901880F991FFC018E
:10153000ED59FA4F80819181AC014F5F5F4FC90136
:10154000880F991FFC01ED59FA4F51834083229671
:101550000FB6F894DEBF0FBECDBFDF91CF910895D7
:101560001F920F920FB60F9211242F933F934F9318
:101570005F936F937F938F939F93AF93BF93EF93FB
:10158000FF93CF93DF93CDB7DEB780E00E94C90908
:10159000DF91CF91FF91EF91BF91AF919F918F918B
:1015A0007F916F915F914F913F912F910F900FBE5F
:1015B0000F901F9018951F920F920FB60F92112443
:1015C0002F933F934F935F936F937F938F939F934B
:1015D000AF93BF93EF93FF93CF93DF93CDB7DEB776
:1015E00081E00E94C909DF91CF91FF91EF91BF91F6
:1015F000AF919F918F917F916F915F914F913F91AB
:101600002F910F900FBE0F901F9018951F920F9261
:101610000FB60F9211242F933F934F935F936F93C5
:101620007F938F939F93AF93BF93EF93FF93CF934A
:10163000DF93CDB7DEB782E00E94C909DF91CF9179
:10164000FF91EF91BF91AF919F918F917F916F919A
:101650005F914F913F912F910F900FBE0F901F9070
:1016600018951F920F920FB60F9211242F933F934C
:101670004F935F936F937F938F939F93AF93BF939A
:10168000EF93FF93CF93DF93CDB7DEB783E00E9454
:10169000C909DF91CF91FF91EF91BF91AF919F91D8
:1016A0008F917F916F915F914F913F912F910F900B
:1016B0000FBE0F901F9018951F920F920FB60F92AA
:1016C00011242F933F934F935F936F937F938F9347
:1016D0009F93AF93BF93EF93FF93CF93DF93CDB7D8
:1016E000DEB780E00E94400ADF91CF91FF91EF9139
:1016F000BF91AF919F918F917F916F915F914F912A
:101700003F912F910F900FBE0F901F9018951F9231
:101710000F920FB60F9211242F933F934F935F9325
:101720006F937F938F939F93AF93BF93EF93FF93A9
:10173000CF93DF93CDB7DEB781E00E94400ADF91FF
:10174000CF91FF91EF91BF91AF919F918F917F9139
:101750006F915F914F913F912F910F900FBE0F901E
:101760001F9018951F920F920FB60F9211242F936E
:101770003F934F935F936F937F938F939F93AF9319
:10178000BF93EF93FF93CF93DF93CDB7DEB782E0A4
:101790000E94400ADF91CF91FF91EF91BF91AF91ED
:1017A0009F918F917F916F915F914F913F912F9179
:1017B0000F900FBE0F901F9018951F920F920FB6AB
:1017C0000F9211242F933F934F935F936F937F93C7
:1017D0008F939F93AF93BF93EF93FF93CF93DF9339
:1017E000CDB7DEB783E00E94400ADF91CF91FF9131
:1017F000EF91BF91AF919F918F917F916F915F9189
:101800004F913F912F910F900FBE0F901F90189501
:10181000CF93DF93CDB7DEB726970FB6F894DEBF30
:101820000FBECDBF9C838B838B819C81039625E06B
:1018300030E0B9010E942A30CB01CC01A0E0B0E039
:10184000880F991FAA1FBB1F880F991FAA1FBB1FB4
:10185000880F991FAA1FBB1F880F991FAA1FBB1FA4
:101860009A8389831E821D8206C02D813E812F5F4F
:101870003F4F3E832D8389819A812D813E81281798
:10188000390798F326960FB6F894DEBF0FBECDBF8A
:10189000DF91CF910895CF93DF93CDB7DEB7219736
:1018A0000FB6F894DEBF0FBECDBF198206C0898186
:1018B0000E94AE0D89818F5F898389818730B8F35B
:1018C0000E94700C0E94860C0E949B0C78942196BA
:1018D0000FB6F894DEBF0FBECDBFDF91CF91089554
:1018E000CF93DF93CDB7DEB785E00E94B10CE6E47D
:1018F000F0E01082AEE6B0E0EEE6F0E080818160DC
:101900008C930E94A50EDF91CF910895CF93DF9322
:10191000CDB7DEB783E00E94CF0CE4E8F0E011829F
:101920001082AFE6B0E0EFE6F0E0808181608C935A
:10193000DF91CF910895CF93DF93CDB7DEB784E0E9
:101940000E94ED0CE2EBF0E01082A0E7B0E0E0E7EF
:10195000F0E0808181608C930E94C50EDF91CF9171
:101960000895CF93DF93CDB7DEB721970FB6F894E4
:10197000DEBF0FBECDBF8983A5E4B0E0E5E4F0E0B3
:101980008081982F987F8981892B8C9321960FB61F
:10199000F894DEBF0FBECDBFDF91CF910895CF93F6
:1019A000DF93CDB7DEB721970FB6F894DEBF0FBE39
:1019B000CDBF8983A1E8B0E0E1E8F0E08081982F15
:1019C000987F8981892B8C9321960FB6F894DEBF7E
:1019D0000FBECDBFDF91CF910895CF93DF93CDB7E9
:1019E000DEB721970FB6F894DEBF0FBECDBF898357
:1019F000A1EBB0E0E1EBF0E08081982F987F898146
:101A0000892B8C9321960FB6F894DEBF0FBECDBF05
:101A1000DF91CF910895CF93DF93CDB7DEB72497B1
:101A20000FB6F894DEBF0FBECDBFE5E4F0E08081D5
:101A3000882F90E087709070880F991F8C519F4F6E
:101A40009C838B83EB81FC81859194919A8389831C
:101A5000FC83EB8389819A8124960FB6F894DEBFCC
:101A60000FBECDBFDF91CF910895CF93DF93CDB758
:101A7000DEB724970FB6F894DEBF0FBECDBFE1E806
:101A8000F0E08081882F90E087709070880F991F18
:101A90008C519F4F9C838B83EB81FC81859194912A
:101AA0009A838983FC83EB8389819A8124960FB67C
:101AB000F894DEBF0FBECDBFDF91CF910895CF93D5
:101AC000DF93CDB7DEB724970FB6F894DEBF0FBE15
:101AD000CDBFE1EBF0E08081882F90E087709070BF
:101AE000880F991F80519F4F9C838B83EB81FC81D2
:101AF000859194919A838983FC83EB8389819A8170
:101B000024960FB6F894DEBF0FBECDBFDF91CF9104
:101B10000895CF93DF93CDB7DEB723970FB6F89430
:101B2000DEBF0FBECDBF89837B836A838981873007
:101B300060F48981882F90E0880F991FFC01E65F8F
:101B4000FA4F8A819B819183808323960FB6F89404
:101B5000DEBF0FBECDBFDF91CF910895CF93DF934E
:101B6000CDB7DEB721970FB6F894DEBF0FBECDBF5D
:101B700089838981873050F48981882F90E0880F8C
:101B8000991FFC01E65FFA4F1182108221960FB671
:101B9000F894DEBF0FBECDBFDF91CF910895EF92D5
:101BA000FF920F931F93CF93DF93CDB7DEB72B97A1
:101BB0000FB6F894DEBF0FBECDBF9B878A87E6E4E1
:101BC000F0E08081898710926F0510927005109265
:101BD0007105109272050E940B0D9C0140E050E0CF
:101BE00080E094E2A4EFB0E0BC01CD010E9473302C
:101BF000DA01C9018D839E83AF83B8878D819E8171
:101C0000AF81B885893B2DE8920726E0A20720E046
:101C1000B20720F58A859B8527E281319207F0F48F
:101C20008A859B85CC01A0E0B0E02D813E814F816B
:101C30005885BC01CD010E940B30DC01CB0128EEA0
:101C400033E040E050E0BC01CD010E945130DA01A8
:101C5000C90189839A83AB83BC833EC08A859B85F7
:101C60007C0100E010E08D819E81AF81B88528EE77
:101C700033E040E050E0BC01CD010E945130DA0178
:101C8000C9019C01AD01C801B7010E940B30DC0104
:101C9000CB0189839A83AB83BC831EC080916F057F
:101CA00090917005A0917105B0917205A3E5B0E027
:101CB000E3E5F0E08081817F8C93A3E5B0E0E3E58C
:101CC000F0E0808181608C938895A3E5B0E0E3E546
:101CD000F0E080818E7F8C9380916F0590917005EC
:101CE000A0917105B09172052227382F492F5A2FE4
:101CF000E6E4F0E08081882F90E0A0E0B0E0790198
:101D00008A01E82AF92A0A2B1B2B8985282F30E023
:101D100040E050E089819A81AB81BC81820F931FA2
:101D2000A41FB51FE816F9060A071B0708F4B6CF6B
:101D30002B960FB6F894DEBF0FBECDBFDF91CF91CB
:101D40001F910F91FF90EF900895CF93DF93CDB740
:101D5000DEB710926B0510926C0510926D05109213
:101D60006E05DF91CF910895CF93DF93CDB7DEB7A6
:101D700080916B0590916C05A0916D05B0916E05F9
:101D8000BC01CD01DF91CF910895CF93DF93CDB703
:101D9000DEB71092730510927405109275051092BB
:101DA0007605DF91CF910895CF93DF93CDB7DEB75E
:101DB0008091730590917405A0917505B091760599
:101DC000BC01CD01DF91CF910895CF93DF93CDB7C3
:101DD000DEB721970FB6F894DEBF0FBECDBF898363
:101DE0008981893079F4A0E8B0E0E0E8F0E0808112
:101DF00082608C93A0E8B0E0E0E8F0E080818E7F24
:101E00008C9320C089818A3079F4A0E8B0E0E0E8C2
:101E1000F0E0808182608C93A0E8B0E0E0E8F0E040
:101E2000808181608C930EC0A0E8B0E0E0E8F0E033
:101E300080818D7F8C93A0E8B0E0E0E8F0E08081C5
:101E400081608C93E8E8F0E011821082EAE8F0E02B
:101E50001182108221960FB6F894DEBF0FBECDBF5F
:101E6000DF91CF910895CF93DF93CDB7DEB722975F
:101E70000FB6F894DEBF0FBECDBF9A838983A0E86A
:101E8000B0E0E0E8F0E080818E7F8C93A0E8B0E0E5
:101E9000E0E8F0E0808182608C93A1E8B0E0E1E8C6
:101EA000F0E0808188608C93A1E8B0E0E1E8F0E0A8
:101EB000808180618C93E6E8F0E089819A8191834A
:101EC0008083E8E8F0E011821082EAE8F0E0118215
:101ED000108222960FB6F894DEBF0FBECDBFDF9101
:101EE000CF910895CF93DF93CDB7DEB7A0E8B0E0F0
:101EF000E0E8F0E080818D7F8C93A0E8B0E0E0E83E
:101F0000F0E080818E7F8C930E94B50F0E94CB0FF2
:101F1000DF91CF910895CF93DF93CDB7DEB7A0E8DF
:101F2000B0E0E0E8F0E0808180688C93A0E8B0E069
:101F3000E0E8F0E080818F7B8C93DF91CF91089572
:101F4000CF93DF93CDB7DEB7A0E8B0E0E0E8F0E0F4
:101F5000808180628C93A0E8B0E0E0E8F0E08081CE
:101F60008F7E8C93DF91CF910895CF93DF93CDB780
:101F7000DEB7A0E8B0E0E0E8F0E090818FE78923E9
:101F80008C93A0E8B0E0E0E8F0E080818F7B8C9358
:101F9000DF91CF910895CF93DF93CDB7DEB7A0E85F
:101FA000B0E0E0E8F0E080818F7D8C93A0E8B0E0C5
:101FB000E0E8F0E080818F7E8C93DF91CF910895EF
:101FC000CF93DF93CDB7DEB722970FB6F894DEBF7D
:101FD0000FBECDBF9A838983E8E8F0E089819A81BA
:101FE0009183808322960FB6F894DEBF0FBECDBFDB
:101FF000DF91CF910895CF93DF93CDB7DEB72297CE
:102000000FB6F894DEBF0FBECDBF9A838983EAE88E
:10201000F0E089819A819183808322960FB6F894AB
:10202000DEBF0FBECDBFDF91CF9108951F920F92FB
:102030000FB60F9211242F933F934F935F936F939B
:102040007F938F939F93AF93BF93EF93FF93CF9320
:10205000DF93CDB7DEB780916B0590916C05A091B1
:102060006D05B0916E050196A11DB11D80936B05A4
:1020700090936C05A0936D05B0936E0580916F05EC
:1020800090917005A0917105B09172050196A11D06
:10209000B11D80936F0590937005A0937105B09367
:1020A000720580910A0590910B05009729F0E09147
:1020B0000A05F0910B051995DF91CF91FF91EF91F2
:1020C000BF91AF919F918F917F916F915F914F9150
:1020D0003F912F910F900FBE0F901F9018951F9258
:1020E0000F920FB60F9211242F933F934F935F934C
:1020F0006F937F938F939F93AF93BF93EF93FF93D0
:10210000CF93DF93CDB7DEB780910C0590910D058D
:10211000009729F0E0910C05F0910D051995DF91DC
:10212000CF91FF91EF91BF91AF919F918F917F914F
:102130006F915F914F913F912F910F900FBE0F9034
:102140001F9018951F920F920FB60F9211242F9384
:102150003F934F935F936F937F938F939F93AF932F
:10216000BF93EF93FF93CF93DF93CDB7DEB780910B
:10217000730590917405A0917505B091760501964F
:10218000A11DB11D8093730590937405A0937505EF
:10219000B09376058091140590911505009729F06C
:1021A000E0911405F09115051995DF91CF91FF91FC
:1021B000EF91BF91AF919F918F917F916F915F91BF
:1021C0004F913F912F910F900FBE0F901F90189538
:1021D0001F920F920FB60F9211242F933F934F939C
:1021E0005F936F937F938F939F93AF93BF93EF937F
:1021F000FF93CF93DF93CDB7DEB780910E0590911B
:102200000F05009729F0E0910E05F0910F05199543
:10221000DF91CF91FF91EF91BF91AF919F918F91FE
:102220007F916F915F914F913F912F910F900FBED2
:102230000F901F9018951F920F920FB60F921124B6
:102240002F933F934F935F936F937F938F939F93BE
:10225000AF93BF93EF93FF93CF93DF93CDB7DEB7E9
:102260008091100590911105009729F0E0911005DB
:10227000F09111051995DF91CF91FF91EF91BF91E9
:10228000AF919F918F917F916F915F914F913F910E
:102290002F910F900FBE0F901F9018951F920F92C5
:1022A0000FB60F9211242F933F934F935F936F9329
:1022B0007F938F939F93AF93BF93EF93FF93CF93AE
:1022C000DF93CDB7DEB7809112059091130500978B
:1022D00029F0E0911205F09113051995DF91CF9146
:1022E000FF91EF91BF91AF919F918F917F916F91EE
:1022F0005F914F913F912F910F900FBE0F901F90C4
:1023000018951F920F920FB60F9211242F933F939F
:102310004F935F936F937F938F939F93AF93BF93ED
:10232000EF93FF93CF93DF93CDB7DEB78091160580
:1023300090911705009729F0E0911605F091170587
:102340001995DF91CF91FF91EF91BF91AF919F913F
:102350008F917F916F915F914F913F912F910F904E
:102360000FBE0F901F9018951F920F920FB60F92ED
:1023700011242F933F934F935F936F937F938F938A
:102380009F93AF93BF93EF93FF93CF93DF93CDB71B
:10239000DEB78091160590911705009729F0E0911E
:1023A0001605F09117051995DF91CF91FF91EF91E7
:1023B000BF91AF919F918F917F916F915F914F915D
:1023C0003F912F910F900FBE0F901F901895CF93B4
:1023D000DF93CDB7DEB722970FB6F894DEBF0FBEFE
:1023E000CDBF9A83898389819A81909319058093BF
:1023F000180522960FB6F894DEBF0FBECDBFDF9151
:10240000CF910895CF93DF93CDB7DEB721970FB665
:10241000F894DEBF0FBECDBF898389818A3031F445
:10242000E0911805F09119058DE01995E0911805D6
:10243000F09119058981199521960FB6F894DEBFA0
:102440000FBECDBFDF91CF910895CF93DF93CDB76E
:10245000DEB722970FB6F894DEBF0FBECDBF9A83CA
:10246000898389819A81009789F00BC0E981FA817B
:10247000208189819A8101969A838983822F0E9483
:102480000212E981FA818081882381F722960FB6B2
:10249000F894DEBF0FBECDBFDF91CF910895CF93EB
:1024A000DF93CDB7DEB72A970FB6F894DEBF0FBE25
:1024B000CDBF9A8389837C836B835E834D8318862B
:1024C0001F8289819A81009709F449C02F8138853C
:1024D00019868B819C812817390710F481E0898740
:1024E0008F819885019698878F8381E099858927C8
:1024F000882391F4E981FA8180818A878A858823FB
:1025000011F091E09A878A8529813A812F5F3F4FA8
:102510003A8329838823D1F618861F8219C0E9815E
:10252000FA818081882361F0E981FA8120818981A3
:102530009A8101969A838983822F0E94021203C096
:1025400080E20E9402128F819885019698878F837E
:102550002F8138858D819E812817390700F32A96AF
:102560000FB6F894DEBF0FBECDBFDF91CF910895B7
:10257000CF93DF93CDB7DEB726970FB6F894DEBFC3
:102580000FBECDBF9D838C838C819D810097B1F060
:1025900003C08E810E9402128C819D819B838A835D
:1025A0008C819D8101969D838C83EA81FB8184913E
:1025B000898389818E838E81882359F726960FB669
:1025C000F894DEBF0FBECDBFDF91CF910895CF93BA
:1025D000DF93CDB7DEB78AE00E940212DF91CF9180
:1025E0000895CF93DF93CDB7DEB724970FB6F89455
:1025F000DEBF0FBECDBF8C838C81882F90E08F70A3
:10260000907080509F4F9B838A83EA81FB818491E5
:10261000898389810E94021224960FB6F894DEBF46
:102620000FBECDBFDF91CF910895CF93DF93CDB78C
:10263000DEB721970FB6F894DEBF0FBECDBF8983FA
:10264000898182958F700E94F11289810E94F11216
:1026500021960FB6F894DEBF0FBECDBFDF91CF91AC
:102660000895CF93DF93CDB7DEB722970FB6F894D6
:10267000DEBF0FBECDBF9A83898389819A81892F5E
:1026800099270E94151389810E94151322960FB66F
:10269000F894DEBF0FBECDBFDF91CF910895CF93E9
:1026A000DF93CDB7DEB724970FB6F894DEBF0FBE29
:1026B000CDBF69837A838B839C8389819A81AB8127
:1026C000BC81CD01AA27BB270E94311389819A8141
:1026D0000E94311324960FB6F894DEBF0FBECDBF13
:1026E000DF91CF910895EF92FF920F931F93CF93B5
:1026F000DF93CDB7DEB7E6970FB6F894DEBF0FBE17
:10270000CDBF8EA76FA748AB29ABEAAAFBAA0CAB3B
:102710001DAB88A98823B1F08AA99BA9ACA9BDA942
:10272000BB2384F48AA99BA9ACA9BDA9B095A095A7
:10273000909581959F4FAF4FBF4F88879987AA8704
:10274000BB8708C08AA99BA9ACA9BDA9888799871E
:10275000AA87BB8788A98EAB8EA9882311F081E058
:102760008EAB9EA98FA5891B81508F83CE010E96BB
:1027700080969D878C878C859D8501979D878C870A
:10278000EC85FD8510828C859D8501979D878C87C2
:102790008EA5282F30E040E050E088859985AA85F5
:1027A000BB85BC01CD010E945130DC01CB018F7093
:1027B000907080509F4F9E838D83ED81FE81849128
:1027C0008C838C81EC85FD8580838EA5282F30E05D
:1027D00040E050E088859985AA85BB85BC01CD0184
:1027E0000E945130DA01C90188879987AA87BB877F
:1027F00047C088859985AA85BB850097A105B10545
:10280000B1F18C859D8501979D878C878EA5282F9A
:1028100030E040E050E088859985AA85BB85BC0101
:10282000CD010E945130DC01CB018F70907080503F
:102830009F4F9B838A83EA81FB818491898389816D
:10284000EC85FD8580838EA5282F30E040E050E0A8
:1028500088859985AA85BB85BC01CD010E94513030
:10286000DA01C90188879987AA87BB8709C08C8547
:102870009D8501979D878C87EC85FD8589A980833F
:102880008F8181508F838F818F3F09F0B2CF88A9CC
:10289000882361F18AA99BA9ACA9BDA9BB2354F4E3
:1028A0008C859D8501979D878C87EC85FD858DE2C4
:1028B00080831CC08AA99BA9ACA9BDA918161906BA
:1028C0001A061B0654F48C859D8501979D878C877D
:1028D000EC85FD858BE2808309C08C859D85019701
:1028E0009D878C87EC85FD8580E280838FA58F8313
:1028F0000BC0EC85FD8520818C859D8501969D878B
:102900008C87822F0E9402128F8181508F838F814A
:102910008F3F79F7E6960FB6F894DEBF0FBECDBFB6
:10292000DF91CF911F910F91FF90EF900895CF937A
:10293000DF93CDB7DEB765970FB6F894DEBF0FBE55
:10294000CDBFCE014E969F878E870BC08D85882385
:1029500029F480E090E09D8B8C8BCBC08D850E940C
:1029600002128B8D882381F08C8D9D8D9E838D83AB
:102970008C8D9D8D01969D8F8C8FED81FE81849134
:102980008C838C818B8B09C0EC8DFD8DE081EB8B72
:102990008C8D9D8D01969D8F8C8F2B892D878D859C
:1029A0008532A1F68B8D882381F08C8D9D8D9B8344
:1029B0008A838C8D9D8D01969D8F8C8FEA81FB8102
:1029C0008491898389818A8B09C0EC8DFD8DE0819A
:1029D000EA8B8C8D9D8D01969D8F8C8F3A893D87DA
:1029E0008D85282F30E0398B288B8889998984360A
:1029F0009105C9F02889398928373105E9F0888996
:102A000099898336910509F00AC02E853F85C90151
:102A100002969F878E87F901808191818D878D85B0
:102A20000E9402129ECF8AE090E098878F8380E117
:102A300097E29A87898708C080E190E098878F8322
:102A400080E090E19A8789872E853F85C9010296AB
:102A50009F878E87F901808191819C878B878D85E7
:102A6000843629F58B859C859923ACF48B859C85D0
:102A7000909581959F4F9C878B878DE20E940212D3
:102A80000AC089859A852AE030E0B9010E942A307F
:102A9000CB019A87898789859A858230910538F09C
:102AA00029853A858B859C858217930750F38B8502
:102AB0009C8529853A85B9010E942A30CB010E9464
:102AC000F1128B859C8529853A85B9010E942A30AF
:102AD0009C878B8789859A852F813885B9010E94CB
:102AE0002A30CB019A87898789859A850097F9F6DC
:102AF00038CF8C899D8965960FB6F894DEBF0FBEDE
:102B0000CDBFDF91CF910895CF93DF93CDB7DEB7DF
:102B1000E0E3F0E01082E1E3F0E01082E7E0F1E0D2
:102B20001082E8E0F1E01082E1E2F0E08FEF8083D4
:102B3000E4E2F0E080E48083E7E2F0E08FEF80837E
:102B4000EAE2F0E08BEF8083EDE2F0E08EEF80834D
:102B5000A3E3B0E0E3E3F0E080818F7D8C93A4E316
:102B6000B0E0E4E3F0E0808180628C93E1E0F1E0AA
:102B70008EEF8083E4E0F1E08EEF8083DF91CF91F0
:102B80000895CF93DF93CDB7DEB724970FB6F894AF
:102B9000DEBF0FBECDBF69837A838B839C830BC05E
:102BA00089819A81AB81BC810197A109B10989838F
:102BB0009A83AB83BC8389819A81AB81BC81009766
:102BC000A105B10569F724960FB6F894DEBF0FBED4
:102BD000CDBFDF91CF910895CF93DF93CDB7DEB70F
:102BE000A5E2B0E0E5E2F0E0808180648C93DF91C3
:102BF000CF910895CF93DF93CDB7DEB7A5E2B0E0D4
:102C0000E5E2F0E080818F7B8C93DF91CF91089596
:102C1000CF93DF93CDB7DEB7E6E4F0E010820E94F9
:102C2000A50EDF91CF910895CF93DF93CDB7DEB797
:102C3000E2E3F0E08081882F90E080729070DF9175
:102C4000CF910895CF93DF93CDB7DEB726970FB618
:102C5000F894DEBF0FBECDBF69837A838B839C83DC
:102C600089819A81AB81BC81BB23CCF089819A8117
:102C7000AB81BC8125E030E040E050E0BC01CD01FB
:102C80000E947330DA01C901880F991FFC01E050DE
:102C9000FE4F0190F081E02DFE83ED832CC08981F1
:102CA0009A81AB81BC81B095A095909581959F4FFD
:102CB000AF4FBF4F25E030E040E050E0BC01CD0118
:102CC0000E947330DA01C9019C01AD0188E490E0F3
:102CD000A0E0B0E0821B930BA40BB50B880F991FEB
:102CE000FC01E050FE4F8081918122273327281B71
:102CF000390B3E832D838D819E8126960FB6F894E5
:102D0000DEBF0FBECDBFDF91CF910895CF93DF938C
:102D1000CDB7DEB726970FB6F894DEBF0FBECDBF96
:102D200069837A838B839C8389819A81AB81BC81FF
:102D30008A559040A040B04089839A83AB83BC837E
:102D400089819A81AB81BC81BB23CCF089819A8136
:102D5000AB81BC8125E030E040E050E0BC01CD011A
:102D60000E947330DA01C901880F991FFC01E050FD
:102D7000FE4F0190F081E02DFE83ED832CC0898110
:102D80009A81AB81BC81B095A095909581959F4F1C
:102D9000AF4FBF4F25E030E040E050E0BC01CD0137
:102DA0000E947330DA01C9019C01AD0188E490E012
:102DB000A0E0B0E0821B930BA40BB50B880F991F0A
:102DC000FC01E050FE4F8081918122273327281B90
:102DD000390B3E832D838D819E8126960FB6F89404
:102DE000DEBF0FBECDBFDF91CF9108950F931F932C
:102DF000CF93DF93CDB7DEB726970FB6F894DEBF3B
:102E00000FBECDBF69837A838B839C8389819A812E
:102E1000AB81BC818A359105A105B10521F189817C
:102E20009A81AB81BC81863A2FEF92072FEFA207E0
:102E30002FEFB207C1F089819A81AB81BC818E30BE
:102E400041E0940740E0A40740E0B40761F08981C5
:102E50009A81AB81BC81823F5EEF95075FEFA5074A
:102E60005FEFB50719F41E821D8224C089819A8103
:102E7000AB81BC81BC01CD010E9486168C01898189
:102E80009A81AB81BC81BC01CD010E9422169C01BC
:102E9000C801B9010E943E30CB019C01220F331FB3
:102EA000C901880F991F880F991FA901480F591F41
:102EB0005E834D838D819E8126960FB6F894DEBF8A
:102EC0000FBECDBFDF91CF911F910F910895CF938A
:102ED000DF93CDB7DEB726970FB6F894DEBF0FBEEF
:102EE000CDBF9E838D831A82198288EF96E00E945F
:102EF000E7110E94CD079C838B838B819C812FEFF0
:102F00008F3F9207B1F326E131E08B819C819F9343
:102F10008F933F932F9381E08F930E9497140F908C
:102F20000F900F900F900F9029813A818B818F70B5
:102F3000F901E758FA4F808389819A8101969A8333
:102F4000898329813A818D819E81281739072CF444
:102F50008B819C818A30910561F681E191E09F939C
:102F60008F9381E08F930E9497140F900F900F9092
:102F700083E00E94460826960FB6F894DEBF0FBE87
:102F8000CDBFDF91CF910895CF93DF93CDB7DEB75B
:102F900080E497E00E94E71189E191E09F938F938D
:102FA00081E08F930E9497140F900F900F9082E012
:102FB00090E00E946717DF91CF910895CF93DF9340
:102FC000CDB7DEB780E497E00E94E7110E94C417F6
:102FD00088E59BE10E94CF0DDF91CF910895CF93BB
:102FE000DF93CDB7DEB780E497E00E94E71183E07E
:102FF0000E9446088EE291E09F938F9381E08F9329
:103000000E9497140F900F900F9083E190E00E9420
:10301000671780918105282F30E084E690E0289F93
:10302000A001299F500D389F500D112480918205D9
:10303000882F90E09C01220F331FC901880F991F30
:10304000880F991F820F931F9A01280F391F8091B3
:103050008305882F90E0820F931F909378058093CB
:10306000770580918505282F30E084E690E0289F41
:10307000A001299F500D389F500D11248091860585
:10308000882F90E09C01220F331FC901880F991FE0
:10309000880F991F820F931F9A01280F391F809163
:1030A0008705882F90E0820F931F9093E20580930D
:1030B000E10580918905282F30E084E690E0289F83
:1030C000A001299F500D389F500D112480918A0531
:1030D000882F90E09C01220F331FC901880F991F90
:1030E000880F991F820F931F9A01280F391F809113
:1030F0008B05882F90E0820F931F9093F8058093A3
:10310000F70588EF96E00E94E7118091F70590910E
:10311000F8052091E1053091E20540917705509145
:1031200078056BE171E09F938F933F932F935F93AB
:103130004F937F936F9381E08F930E9497148DB785
:103140009EB709960FB6F8949EBF0FBE8DBFDF9154
:10315000CF910895EF92FF920F931F93CF93DF9338
:10316000CDB7DEB788EF96E00E94E7118091770532
:10317000909178054097AA2797FDA095BA2FBC019A
:10318000CD010E941C2FDC01CB0124EF3DEF44E96F
:103190005FE3BC01CD010E94A82FDC01CB017C01C3
:1031A0008D018091F7059091F80580589040AA27ED
:1031B00097FDA095BA2FBC01CD010E941C2FDC0108
:1031C000CB012AEB39E44CEC5FE3BC01CD010E945A
:1031D000A82FDC01CB019C01AD01C801B7010E9401
:1031E000852EDC01CB01BC01CD010E94E92EDC0162
:1031F000CB01909300068093FF0580917705909115
:1032000078054097AA2797FDA095BA2FBC01CD015C
:103210000E941C2FDC01CB0124EF3DEF44E95FE36A
:10322000BC01CD010E94A82FDC01CB017C018D01E6
:103230008091F7059091F80580589040AA2797FD56
:10324000A095BA2FBC01CD010E941C2FDC01CB013F
:1032500025EC30E240E55FEBBC01CD010E94A82FD8
:10326000DC01CB019C01AD01C801B7010E94852E94
:10327000DC01CB017C018D018091E1059091E2059B
:1032800080589040AA2797FDA095BA2FBC01CD0188
:103290000E941C2FDC01CB0127E231E348EC5EEBFE
:1032A000BC01CD010E94A82FDC01CB019C01AD0126
:1032B000C801B7010E94852EDC01CB01BC01CD0104
:1032C0000E94E92EDC01CB019093F0058093EF057D
:1032D00080917705909178054097AA2797FDA09552
:1032E000BA2FBC01CD010E941C2FDC01CB0124EFC1
:1032F0003DEF44E95FE3BC01CD010E94A82FDC0152
:10330000CB017C018D018091E1059091E20580580F
:103310009040AA2797FDA095BA2FBC01CD010E942D
:103320001C2FDC01CB0129EE36E241E050E4BC0168
:10333000CD010E94A82FDC01CB019C01AD01C80189
:10334000B7010E94852EDC01CB01BC01CD010E949A
:10335000E92EDC01CB019093E6058093E505809191
:10336000E5059091E6052091EF053091F00540913B
:10337000FF055091000661E371E09F938F933F93A7
:103380002F935F934F937F936F9381E08F930E946E
:1033900097148DB79EB709960FB6F8949EBF0FBECF
:1033A0008DBFDF91CF911F910F91FF90EF90089506
:1033B000CF92DF92EF92FF920F931F93CF93DF9301
:1033C000CDB7DEB72E970FB6F894DEBF0FBECDBFD8
:1033D0009A8389837C836B835E834D8338872F83B5
:1033E0001A870987FC86EB86DE86CD8680E497E027
:1033F0000E94E71183E00E9446082FE931E08981AD
:103400009A819F938F933F932F9381E08F930E9494
:1034100097140F900F900F900F900F908B819C81BD
:1034200024E630E0B9010E943E302AE030E0B901E4
:103430000E943E308C018B819C8124E630E0B901F2
:103440000E943E302AE030E0B9010E943E30CB01BC
:10345000FC018B819C8124E630E0B9010E943E3062
:10346000CB0128E931E01F930F93FF93EF939F93D4
:103470008F933F932F9381E08F930E9497148DB782
:103480009EB709960FB6F8949EBF0FBE8DBF8D8173
:103490009E8124E630E0B9010E943E302AE030E00F
:1034A000B9010E943E308C018D819E8124E630E07E
:1034B000B9010E943E302AE030E0B9010E943E305E
:1034C000CB01FC018D819E8124E630E0B9010E9490
:1034D0003E30CB0121E931E01F930F93FF93EF932F
:1034E0009F938F933F932F9381E08F930E94971424
:1034F0008DB79EB709960FB6F8949EBF0FBE8DBFCD
:103500008F81988524E630E0B9010E943E302AE0A0
:1035100030E0B9010E943E308C018F81988524E60D
:1035200030E0B9010E943E302AE030E0B9010E944B
:103530003E30CB01FC018F81988524E630E0B90153
:103540000E943E30CB012AE831E01F930F93FF9396
:10355000EF939F938F933F932F9381E08F930E94DC
:1035600097148DB79EB709960FB6F8949EBF0FBEFD
:103570008DBF89859A8524E630E0B9010E943E30EE
:103580002AE030E0B9010E943E308C0189859A859D
:1035900024E630E0B9010E943E302AE030E0B90173
:1035A0000E943E30CB01FC0189859A8524E630E0FB
:1035B000B9010E943E30CB0123E831E01F930F9305
:1035C000FF93EF939F938F933F932F9381E08F937C
:1035D0000E9497148DB79EB709960FB6F8949EBFB8
:1035E0000FBE8DBF8B859C8524E630E0B9010E941B
:1035F0003E302AE030E0B9010E943E308C018B85DC
:103600009C8524E630E0B9010E943E302AE030E09B
:10361000B9010E943E30CB01FC018B859C8524E6DC
:1036200030E0B9010E943E30CB012CE731E01F931E
:103630000F93FF93EF939F938F933F932F9381E08B
:103640008F930E9497148DB79EB709960FB6F89482
:103650009EBF0FBE8DBF8D859E8524E630E0B901EB
:103660000E943E302AE030E0B9010E943E308C01D9
:103670008D859E8524E630E0B9010E943E302AE027
:1036800030E0B9010E943E30CB01FC018D859E8562
:1036900024E630E0B9010E943E30CB0125E731E05D
:1036A0001F930F93FF93EF939F938F933F932F93CA
:1036B00081E08F930E9497148DB79EB709960FB63D
:1036C000F8949EBF0FBE8DBF86E090E00E94671702
:1036D00088EF96E00E94E71120E731E089819A8126
:1036E0009F938F933F932F9381E08F930E94971422
:1036F0000F900F900F900F900F908B819C8124E67C
:1037000030E0B9010E943E302AE030E0B9010E9469
:103710003E308C018B819C8124E630E0B9010E940F
:103720003E302AE030E0B9010E943E30CB01FC017E
:103730008B819C8124E630E0B9010E943E30CB01B0
:1037400029E631E01F930F93FF93EF939F938F939D
:103750003F932F9381E08F930E9497148DB79EB76C
:1037600009960FB6F8949EBF0FBE8DBF8D819E81C6
:1037700024E630E0B9010E943E302AE030E0B90191
:103780000E943E308C018D819E8124E630E0B9019B
:103790000E943E302AE030E0B9010E943E30CB0169
:1037A000FC018D819E8124E630E0B9010E943E300B
:1037B000CB0122E631E01F930F93FF93EF939F938A
:1037C0008F933F932F9381E08F930E9497148DB72F
:1037D0009EB709960FB6F8949EBF0FBE8DBF8F811E
:1037E000988524E630E0B9010E943E302AE030E0BE
:1037F000B9010E943E308C018F81988524E630E02B
:10380000B9010E943E302AE030E0B9010E943E300A
:10381000CB01FC018F81988524E630E0B9010E943C
:103820003E30CB012BE531E01F930F93FF93EF93D5
:103830009F938F933F932F9381E08F930E949714D0
:103840008DB79EB709960FB6F8949EBF0FBE8DBF79
:1038500089859A8524E630E0B9010E943E302AE04D
:1038600030E0B9010E943E308C0189859A8524E6BA
:1038700030E0B9010E943E302AE030E0B9010E94F8
:103880003E30CB01FC0189859A8524E630E0B90100
:103890000E943E30CB0124E531E01F930F93FF934C
:1038A000EF939F938F933F932F9381E08F930E9489
:1038B00097148DB79EB709960FB6F8949EBF0FBEAA
:1038C0008DBF8B859C8524E630E0B9010E943E3097
:1038D0002AE030E0B9010E943E308C018B859C8546
:1038E00024E630E0B9010E943E302AE030E0B90120
:1038F0000E943E30CB01FC018B859C8524E630E0A4
:10390000B9010E943E30CB012DE431E01F930F93AB
:10391000FF93EF939F938F933F932F9381E08F9328
:103920000E9497148DB79EB709960FB6F8949EBF64
:103930000FBE8DBF8D859E8524E630E0B9010E94C3
:103940003E302AE030E0B9010E943E308C018D8586
:103950009E8524E630E0B9010E943E302AE030E046
:10396000B9010E943E30CB01FC018D859E8524E685
:1039700030E0B9010E943E30CB0124E431E01F93D6
:103980000F93FF93EF939F938F933F932F9381E038
:103990008F930E9497148DB79EB709960FB6F8942F
:1039A0009EBF0FBE8DBF2E960FB6F894DEBF0FBE22
:1039B000CDBFDF91CF911F910F91FF90EF90DF90DE
:1039C000CF9008950F931F93CF93DF93CDB7DEB7BA
:1039D00026970FB6F894DEBF0FBECDBF9A838983BA
:1039E00080E497E00E94E71183E00E94460826EEFB
:1039F00031E089819A819F938F933F932F9381E048
:103A00008F930E9497140F900F900F900F900F902C
:103A100083E690E00E94671780917F05282F30E0B1
:103A200084E690E0289FA001299F500D389F500DFB
:103A3000112480918005882F90E09C01220F331F74
:103A4000C901880F991F880F991F820F931F9A0130
:103A5000280F391F80918105882F90E0820F931FD6
:103A60009093F6058093F50580918305282F30E02B
:103A700084E690E0289FA001299F500D389F500DAB
:103A8000112480918405882F90E09C01220F331F20
:103A9000C901880F991F880F991F820F931F9A01E0
:103AA000280F391F80918505882F90E0820F931F82
:103AB0009093E8058093E70580918705282F30E0F3
:103AC00084E690E0289FA001299F500D389F500D5B
:103AD000112480918805882F90E09C01220F331FCC
:103AE000C901880F991F880F991F820F931F9A0190
:103AF000280F391F80918905882F90E0820F931F2E
:103B00009093E4058093E30580918B05282F30E0A6
:103B100084E690E0289FA001299F500D389F500D0A
:103B2000112480918C05882F90E09C01220F331F77
:103B3000C901880F991F880F991F820F931F9A013F
:103B4000280F391F80918D05882F90E0820F931FD9
:103B50009093EC058093EB0580919205282F30E03F
:103B600088EE93E0289FA001299F500D389F500DAB
:103B7000112480919305282F30E084E690E0BC0169
:103B8000269FC001279F900D369F900D1124480F4E
:103B9000591F80919405882F90E09C01220F331FBC
:103BA000C901880F991F880F991F820F931F9A01CF
:103BB000280F391F80919505882F90E0820F931F61
:103BC000AA2797FDA095BA2F8093DD059093DE0577
:103BD000A093DF05B093E0052091F5053091F6053F
:103BE0008091E7059091E805820F931F9C838B835A
:103BF0008B819C81992334F46B817C816F5F7F4F33
:103C00007C836B838B819C81959587959093FA0536
:103C10008093F9052091E3053091E4058091EB054F
:103C20009091EC05820F931F9E838D838D819E81E1
:103C3000992334F46D817E816F5F7F4F7E836D8326
:103C40008D819E81959587959093EA058093E905EE
:103C500088EF96E00E94E7118091DD059091DE05E6
:103C6000A091DF05B091E0052091EB053091EC05C6
:103C70004091E3055091E4056091E7057091E805F6
:103C8000E091F505F091F60504EB11E0BF93AF93D9
:103C90009F938F933F932F935F934F937F936F9354
:103CA000FF93EF931F930F9381E08F930E949714DC
:103CB0008DB79EB70F960FB6F8949EBF0FBE8DBFFF
:103CC0008091E9059091EA052091F9053091FA0576
:103CD00044EA51E09F938F933F932F935F934F93C9
:103CE00081E08F930E9497146DB77EB7695F7F4F15
:103CF0000FB6F8947EBF0FBE6DBF26960FB6F89430
:103D0000DEBF0FBECDBFDF91CF911F910F91089500
:103D1000CF93DF93CDB7DEB722970FB6F894DEBF0F
:103D20000FBECDBF9A838983A2E0B1E0E2E0F1E06B
:103D3000808184608C938091BE029091BF029C012F
:103D4000220F331F220F331F220F331F84ED93E006
:103D5000AC01421B530B9A0189819A81A901481B2E
:103D6000590BCA01AA2797FDA095BA2FBC01CD0116
:103D70000E94C115A2E0B1E0E2E0F1E080818B7F1A
:103D80008C93A8E2B0E0E8E2F0E0808181608C935F
:103D90008091BE029091BF029C01220F331F220F1F
:103DA000331F220F331F84ED93E0AC01421B530BF2
:103DB0009A0189819A81820F931FAA2797FDA09566
:103DC000BA2FBC01CD010E94C115A8E2B0E0E8E223
:103DD000F0E080818E7F8C9322960FB6F894DEBF40
:103DE0000FBECDBFDF91CF910895CF93DF93CDB7B5
:103DF000DEB728970FB6F894DEBF0FBECDBF9E8307
:103E00008D8378876F8383E190E09C838B8387E148
:103E100090E09A8389838091BE029091BF029C01B9
:103E2000285230408B819C81AC01249FC001259F8A
:103E3000900D349F900D1124805E9C4FAA2797FD12
:103E4000A095BA2F8093FB059093FC05A093FD05E8
:103E5000B093FE058091C0029091C1029C01205256
:103E6000304089819A81AC01249FC001259F900D2B
:103E7000349F900D112482529C4FAA2797FDA09544
:103E8000BA2F8093F1059093F205A093F305B093B8
:103E9000F4058D819E819C01442737FD4095542F68
:103EA0008091DD059091DE05A091DF05B091E005E0
:103EB000281739074A075B070CF080C08091E70597
:103EC0009091E805813591050CF078C08091EB0563
:103ED0009091EC05813491050CF070C0A8E2B0E03F
:103EE000E8E2F0E0808180628C938091FB05909104
:103EF000FC05A091FD05B091FE05BC01CD010E941D
:103F0000C115A8E2B0E0E8E2F0E080818F7D8C93FB
:103F1000A8E2B0E0E8E2F0E0808182608C9368EF94
:103F200072E080E090E00E94C115A8E2B0E0E8E213
:103F3000F0E080818D7F8C938F8198859C0121504A
:103F400030408091BE029091BF02A901489F90012C
:103F5000499F300D589F300D11248091F9059091A3
:103F6000FA05820F931F2F813885B9010E943E30D8
:103F7000CB019093BF028093BE028F8198859C01F4
:103F8000215030408091C0029091C102A901489F08
:103F90009001499F300D589F300D11248091E90503
:103FA0009091EA05820F931F2F813885B9010E94F5
:103FB0003E30CB019093C1028093C00228960FB689
:103FC000F894DEBF0FBECDBFDF91CF910895CF93A0
:103FD000DF93CDB7DEB7AEE2B0E0EEE2F0E0808195
:103FE00088608C936FED72E080E090E00E94C115D4
:103FF000AEE2B0E0EEE2F0E08081877F8C93A2E059
:10400000B1E0E2E0F1E0808180618C9360E674E0F1
:1040100080E090E00E94C115A2E0B1E0E2E0F1E0B2
:1040200080818F7E8C93AEE2B0E0EEE2F0E08081A2
:1040300080628C936AE971E080E090E00E94C11593
:10404000AEE2B0E0EEE2F0E080818F7D8C93DF9114
:10405000CF910895CF93DF93CDB7DEB7A2E2B0E062
:10406000E2E2F0E0808180618C936AE872E080E0B7
:1040700090E00E94C115A2E2B0E0E2E2F0E08081AF
:104080008F7E8C93A2E0B1E0E2E0F1E08081806479
:104090008C9368E671E080E090E00E94C115A2E098
:1040A000B1E0E2E0F1E080818F7B8C93A8E2B0E0A8
:1040B000E8E2F0E0808184608C9365EC73E080E05E
:1040C00090E00E94C115A8E2B0E0E8E2F0E0808153
:1040D0008B7F8C93A2E2B0E0E2E2F0E08081886026
:1040E0008C9366E272E080E090E00E94C115A2E24B
:1040F000B0E0E2E2F0E08081877F8C93DF91CF91A6
:104100000895CF93DF93CDB7DEB7A2E2B0E0E2E24D
:10411000F0E0808188608C9366EB73E080E090E053
:104120000E94C115A2E2B0E0E2E2F0E08081877F68
:104130008C93DF91CF910895CF93DF93CDB7DEB706
:10414000A2E2B0E0E2E2F0E0808188608C9360E976
:1041500071E080E090E00E94C115A2E2B0E0E2E2EE
:10416000F0E08081877F8C93DF91CF910895CF938A
:10417000DF93CDB7DEB7A2E2B0E0E2E2F0E080810B
:1041800088608C9366E272E080E090E00E94C11546
:10419000A2E2B0E0E2E2F0E08081877F8C93DF91E1
:1041A000CF910895CF93DF93CDB7DEB7A2E0B1E012
:1041B000E2E0F1E0808184608C936CE474E080E064
:1041C00090E00E94C115A2E0B1E0E2E0F1E0808160
:1041D0008B7F8C93A8E2B0E0E8E2F0E08081816020
:1041E0008C936CE474E080E090E00E94C115A8E23A
:1041F000B0E0E8E2F0E080818E7F8C93DF91CF9198
:104200000895CF93DF93CDB7DEB7A2E0B1E0E2E04F
:10421000F1E0808184608C9360E971E080E090E05F
:104220000E94C115A2E0B1E0E2E0F1E080818B7F65
:104230008C93A8E2B0E0E8E2F0E0808181608C93AA
:1042400060E971E080E090E00E94C115A8E2B0E072
:10425000E8E2F0E080818E7F8C93DF91CF9108952A
:10426000CF93DF93CDB7DEB7A2E0B1E0E2E0F1E0BB
:10427000808184608C9360E971E080E090E00E942E
:10428000C115A2E0B1E0E2E0F1E080818B7F8C9388
:10429000A8E2B0E0E8E2F0E0808181608C936CE419
:1042A00074E080E090E00E94C115A8E2B0E0E8E28E
:1042B000F0E080818E7F8C93DF91CF910895CF9332
:1042C000DF93CDB7DEB7A2E0B1E0E2E0F1E08081BC
:1042D00084608C936CE474E080E090E00E94C115EF
:1042E000A2E0B1E0E2E0F1E080818B7F8C93A8E274
:1042F000B0E0E8E2F0E0808181608C9360E971E0F9
:1043000080E090E00E94C115A8E2B0E0E8E2F0E0B1
:1043100080818E7F8C93DF91CF910895CF93DF932F
:10432000CDB7DEB7A2E0B1E0E2E0F1E080818460E9
:104330008C936CEB72E080E090E00E94C115A2E0EB
:10434000B1E0E2E0F1E080818B7F8C93A8E2B0E005
:10435000E8E2F0E0808181608C936CEB72E080E0B9
:1043600090E00E94C115A8E2B0E0E8E2F0E08081B0
:104370008E7F8C93DF91CF910895CF93DF93CDB74C
:10438000DEB7A8E2B0E0E8E2F0E0808180628C93E2
:104390006AED72E080E090E00E94C115A8E2B0E012
:1043A000E8E2F0E080818F7D8C93A8E2B0E0E8E263
:1043B000F0E0808182608C936EED73E080E090E0AD
:1043C0000E94C115A8E2B0E0E8E2F0E080818D7FB4
:1043D0008C93DF91CF910895CF93DF93CDB7DEB764
:1043E00024970FB6F894DEBF0FBECDBF1C821B8290
:1043F0001A8219821C821B8233C0A8E2B0E0E8E274
:10440000F0E0808180628C9364E873E080E090E06B
:104410000E94C115A8E2B0E0E8E2F0E080818F7D63
:104420008C93A8E2B0E0E8E2F0E0808182608C93B7
:1044300066E074E080E090E00E94C115A8E2B0E080
:10444000E8E2F0E080818D7F8C9368E873E180E0A2
:1044500090E00E94C1158B819C8101969C838B8387
:104460008B819C818830910544F21C821B8247C05D
:10447000A2E2B0E0E2E2F0E0808180618C9362E54C
:1044800073E080E090E00E94C115A2E2B0E0E2E2B9
:10449000F0E080818F7E8C93A2E0B1E0E2E0F1E079
:1044A000808180648C9368EE73E080E090E00E94ED
:1044B000C115A2E0B1E0E2E0F1E080818F7B8C9356
:1044C000A8E2B0E0E8E2F0E0808184608C9364EFE1
:1044D00071E080E090E00E94C115A8E2B0E0E8E25F
:1044E000F0E080818B7F8C9368E873E180E090E05E
:1044F0000E94C1158B819C8101969C838B838B814B
:104500009C81883291050CF4B3CF1C821B822FC092
:104510001A8219820DC00E94812060E777E180E055
:1045200090E00E94C11589819A8101969A838983BE
:1045300089819A818A30910574F31A8219820DC09B
:104540000E949C2060E777E180E090E00E94C11526
:1045500089819A8101969A83898389819A818A3097
:10456000910574F38B819C8101969C838B838B8155
:104570009C818F30910564F21C821B820DC00E94C9
:104580002A2068E873E180E090E00E94C1158B81E9
:104590009C8101969C838B838B819C8188329105C1
:1045A00074F31C821B820DC00E94BD2168E873E178
:1045B00080E090E00E94C1158B819C8101969C83D4
:1045C0008B838B819C818830910574F324960FB680
:1045D000F894DEBF0FBECDBFDF91CF910895CF938A
:1045E000DF93CDB7DEB7A8E2B0E0E8E2F0E080818B
:1045F00080628C936CE073E080E090E00E94C115D3
:10460000A8E2B0E0E8E2F0E080818F7D8C93A8E240
:10461000B0E0E8E2F0E0808182608C9364E873E0CF
:1046200080E090E00E94C115A8E2B0E0E8E2F0E08E
:1046300080818D7F8C93AEE2B0E0EEE2F0E080818D
:1046400088608C9364E873E080E090E00E94C1157C
:10465000AEE2B0E0EEE2F0E08081877F8C93A2E0F2
:10466000B1E0E2E0F1E0808180618C9368E671E086
:1046700080E090E00E94C115A2E0B1E0E2E0F1E04C
:1046800080818F7E8C93AEE2B0E0EEE2F0E080813C
:1046900080628C9360EC73E080E090E00E94C11532
:1046A000AEE2B0E0EEE2F0E080818F7D8C93A2E29A
:1046B000B0E0E2E2F0E0808180618C9364EF71E031
:1046C00080E090E00E94C115A2E2B0E0E2E2F0E0FA
:1046D00080818F7E8C93A2E0B1E0E2E0F1E0808106
:1046E00080648C9360E674E080E090E00E94C115E5
:1046F000A2E0B1E0E2E0F1E080818F7B8C93A8E260
:10470000B0E0E8E2F0E0808184608C9368E671E0DC
:1047100080E090E00E94C115A8E2B0E0E8E2F0E09D
:1047200080818B7F8C93A2E2B0E0E2E2F0E08081B6
:1047300088608C9366E272E080E090E00E94C11590
:10474000A2E2B0E0E2E2F0E08081877F8C93DF912B
:10475000CF910895CF93DF93CDB7DEB70E94E71FC7
:104760000E942A200E94BD21DF91CF910895CF930E
:10477000DF93CDB7DEB7AEE2B0E0EEE2F0E08081ED
:1047800088608C9368EE73E080E090E00E94C11531
:10479000AEE2B0E0EEE2F0E08081877F8C93A2E0B1
:1047A000B1E0E2E0F1E0808180618C9360E273E04F
:1047B00080E090E00E94C115A2E0B1E0E2E0F1E00B
:1047C00080818F7E8C93AEE2B0E0EEE2F0E08081FB
:1047D00080628C936AE971E080E090E00E94C115EC
:1047E000AEE2B0E0EEE2F0E080818F7D8C93A2E259
:1047F000B0E0E2E2F0E0808180618C9364EF71E0F0
:1048000080E090E00E94C115A2E2B0E0E2E2F0E0B8
:1048100080818F7E8C93A2E0B1E0E2E0F1E08081C4
:1048200080648C9368E572E080E090E00E94C1159E
:10483000A2E0B1E0E2E0F1E080818F7B8C93A8E21E
:10484000B0E0E8E2F0E0808184608C9365EC73E096
:1048500080E090E00E94C115A8E2B0E0E8E2F0E05C
:1048600080818B7F8C93A2E2B0E0E2E2F0E0808175
:1048700088608C9364EF71E080E090E00E94C11545
:10488000A2E2B0E0E2E2F0E08081877F8C93DF91EA
:10489000CF910895CF93DF93CDB7DEB7AEE2B0E00E
:1048A000EEE2F0E0808188608C9368EE73E080E057
:1048B00090E00E94C115AEE2B0E0EEE2F0E080814F
:1048C000877F8C93A2E0B1E0E2E0F1E0808180613B
:1048D0008C9364E873E080E090E00E94C115A2E050
:1048E000B1E0E2E0F1E080818F7E8C93AEE2B0E057
:1048F000EEE2F0E0808180628C936AE971E080E012
:1049000090E00E94C115AEE2B0E0EEE2F0E08081FE
:104910008F7D8C93A2E2B0E0E2E2F0E080818061E2
:104920008C9364EF71E080E090E00E94C115A2E2F8
:10493000B0E0E2E2F0E080818F7E8C93A2E0B1E013
:10494000E2E0F1E0808180648C9364EF71E080E0CC
:1049500090E00E94C115A2E0B1E0E2E0F1E08081C8
:104960008F7B8C93A8E2B0E0E8E2F0E08081846085
:104970008C9365EC73E080E090E00E94C115A8E2A2
:10498000B0E0E8E2F0E080818B7F8C93A2E2B0E0BF
:10499000E2E2F0E0808188608C9364EF71E080E077
:1049A00090E00E94C115A2E2B0E0E2E2F0E0808176
:1049B000877F8C93DF91CF910895CF93DF93CDB70D
:1049C000DEB7AEE2B0E0EEE2F0E0808188608C938A
:1049D0006CEB72E080E090E00E94C115AEE2B0E0C6
:1049E000EEE2F0E08081877F8C93A2E0B1E0E2E02C
:1049F000F1E0808180618C9364E873E080E090E076
:104A00000E94C115A2E0B1E0E2E0F1E080818F7E7A
:104A10008C93AEE2B0E0EEE2F0E0808180628C93B5
:104A20006AE971E080E090E00E94C115AEE2B0E07A
:104A3000EEE2F0E080818F7D8C93A2E2B0E0E2E2D2
:104A4000F0E0808180618C9360E273E080E090E030
:104A50000E94C115A2E2B0E0E2E2F0E080818F7E28
:104A60008C93A2E0B1E0E2E0F1E0808180648C937D
:104A700064EF71E080E090E00E94C115A2E0B1E037
:104A8000E2E0F1E080818F7B8C93A8E2B0E0E8E285
:104A9000F0E0808184608C9365EC73E080E090E0CE
:104AA0000E94C115A8E2B0E0E8E2F0E080818B7FCF
:104AB0008C93A2E2B0E0E2E2F0E0808188608C9327
:104AC00064EF71E080E090E00E94C115A2E2B0E0E6
:104AD000E2E2F0E08081877F8C93DF91CF910895AF
:104AE000CF93DF93CDB7DEB724970FB6F894DEBF30
:104AF0000FBECDBF1C821B821A8219821C821B82B0
:104B00002FC01A8219820DC00E944A2460E777E103
:104B100080E090E00E94C11589819A8101969A8374
:104B2000898389819A818931910574F31A82198266
:104B30000DC00E94DD2460E777E180E090E00E94F4
:104B4000C11589819A8101969A83898389819A8185
:104B50008931910574F38B819C8101969C838B83B1
:104B60008B819C818430910564F224960FB6F89471
:104B7000DEBF0FBECDBFDF91CF910895CF93DF93FE
:104B8000CDB7DEB7AEE2B0E0EEE2F0E08081886063
:104B90008C9368EE73E080E090E00E94C115AEE275
:104BA000B0E0EEE2F0E08081877F8C93A2E0B1E09C
:104BB000E2E0F1E0808180618C9364E873E080E062
:104BC00090E00E94C115A2E0B1E0E2E0F1E0808156
:104BD0008F7E8C93AEE2B0E0EEE2F0E08081806206
:104BE0008C936AE971E080E090E00E94C115AEE22A
:104BF000B0E0EEE2F0E080818F7D8C93A2E2B0E045
:104C0000E2E2F0E0808180618C9364EF71E080E00B
:104C100090E00E94C115A2E2B0E0E2E2F0E0808103
:104C20008F7E8C93A2E0B1E0E2E0F1E080818064CD
:104C30008C9364EF71E080E090E00E94C115A2E0E7
:104C4000B1E0E2E0F1E080818F7B8C93A8E2B0E0FC
:104C5000E8E2F0E0808184608C9365EC73E080E0B2
:104C600090E00E94C115A8E2B0E0E8E2F0E08081A7
:104C70008B7F8C93A2E2B0E0E2E2F0E0808188607A
:104C80008C9364EF71E080E090E00E94C115A2E295
:104C9000B0E0E2E2F0E08081877F8C93DF91CF91FA
:104CA0000895CF93DF93CDB7DEB7AEE2B0E0EEE28A
:104CB000F0E0808188608C9368EE73E080E090E0A3
:104CC0000E94C115AEE2B0E0EEE2F0E08081877FA5
:104CD0008C93A2E0B1E0E2E0F1E0808180618C930E
:104CE00060E674E080E090E00E94C115A2E0B1E0CF
:104CF000E2E0F1E080818F7E8C93AEE2B0E0EEE204
:104D0000F0E0808180628C936AE971E080E090E05D
:104D10000E94C115AEE2B0E0EEE2F0E080818F7D4E
:104D20008C93A2E2B0E0E2E2F0E0808180618C93BB
:104D300064EF71E080E090E00E94C115A2E2B0E073
:104D4000E2E2F0E080818F7E8C93A2E0B1E0E2E0CD
:104D5000F1E0808180648C9368E671E080E090E00F
:104D60000E94C115A2E0B1E0E2E0F1E080818F7B1A
:104D70008C93A8E2B0E0E8E2F0E0808184608C935C
:104D800065EC73E080E090E00E94C115A8E2B0E01D
:104D9000E8E2F0E080818B7F8C93A2E2B0E0E2E277
:104DA000F0E0808188608C9364EF71E080E090E0B7
:104DB0000E94C115A2E2B0E0E2E2F0E08081877FCC
:104DC0008C93DF91CF910895CF93DF93CDB7DEB76A
:104DD00024970FB6F894DEBF0FBECDBF1C821B8296
:104DE0001A8219821C821B822FC01A8219820DC05E
:104DF0000E94BE2560E777E180E090E00E94C11547
:104E000089819A8101969A83898389819A818931DE
:104E1000910574F31A8219820DC00E94512660E731
:104E200077E180E090E00E94C11589819A81019626
:104E30009A83898389819A818931910574F38B8161
:104E40009C8101969C838B838B819C81843091050E
:104E500064F224960FB6F894DEBF0FBECDBFDF918B
:104E6000CF910895CF93DF93CDB7DEB70E943B2754
:104E7000DF91CF910895CF93DF93CDB7DEB722971F
:104E80000FB6F894DEBF0FBECDBF1A8219821A8208
:104E900019820DC00E94AA2368E873E180E090E0C7
:104EA0000E94C11589819A8101969A83898389819B
:104EB0009A818832910574F31A8219820BC06CEDC5
:104EC0007FEF80E090E00E94C11589819A81019670
:104ED0009A83898389819A818C30910584F31A821F
:104EE00019820DC00E94EF2268E873E180E090E033
:104EF0000E94C11589819A8101969A83898389814B
:104F00009A818832910574F31A8219820BC06CED74
:104F10007FEF80E090E00E94C11589819A8101961F
:104F20009A83898389819A818C30910584F30E94C8
:104F3000EC211A8219820BC06CED7FEF80E090E0CB
:104F40000E94C11589819A8101969A8389838981FA
:104F50009A818C30910584F322960FB6F894DEBFC7
:104F60000FBECDBFDF91CF910895CF93DF93CDB723
:104F7000DEB70E94FA150E941416009711F00E94E5
:104F8000EC15E0E3F0E08FEF8083E7E0F1E08FEFF6
:104F90008083A2E0B1E0E2E0F1E0808180648C9364
:104FA000A2E0B1E0E2E0F1E0808180628C93A2E0D7
:104FB000B1E0E2E0F1E0808180618C93A2E0B1E0B9
:104FC000E2E0F1E0808188608C93A2E0B1E0E2E071
:104FD000F1E0808184608C93AEE2B0E0EEE2F0E03C
:104FE000808180688C93AEE2B0E0EEE2F0E08081F8
:104FF00080648C93AEE2B0E0EEE2F0E0808180620B
:105000008C93AEE2B0E0EEE2F0E0808180618C93C0
:10501000AEE2B0E0EEE2F0E0808188608C93AEE238
:10502000B0E0EEE2F0E0808184608C93A8E2B0E032
:10503000E8E2F0E0808181608C93A8E2B0E0E8E2F1
:10504000F0E0808182608C93A8E2B0E0E8E2F0E0DA
:10505000808184608C93A8E2B0E0E8E2F0E0808197
:1050600088608C93A8E2B0E0E8E2F0E080818061A3
:105070008C93A8E2B0E0E8E2F0E0808180628C935B
:10508000A8E2B0E0E8E2F0E0808180648C93A8E2DE
:10509000B0E0E8E2F0E0808180688C93A5E0B1E0C8
:1050A000E5E0F1E0808180648C93A2E2B0E0E2E28E
:1050B000F0E0808180688C93A2E2B0E0E2E2F0E070
:1050C000808180648C93A2E2B0E0E2E2F0E0808133
:1050D00080628C93A2E2B0E0E2E2F0E08081806145
:1050E0008C93A2E2B0E0E2E2F0E0808188608C93F1
:1050F000A2E2B0E0E2E2F0E0808184608C93A2E280
:10510000B0E0E2E2F0E0808182608C93A2E2B0E065
:10511000E2E2F0E0808181608C93A1E3B0E0E1E322
:10512000F0E0808181608C93A1E3B0E0E1E3F0E006
:10513000808182608C93A1E3B0E0E1E3F0E08081C4
:1051400084608C93A1E3B0E0E1E3F0E080818860CB
:105150008C93A1E3B0E0E1E3F0E0808180618C9387
:10516000A1E3B0E0E1E3F0E0808180628C93A1E311
:10517000B0E0E1E3F0E0808180648C93A1E3B0E0F3
:10518000E1E3F0E0808180688C93A8E0B1E0E8E0A2
:10519000F1E0808181608C93A8E0B1E0E8E0F1E08B
:1051A000808182608C93A8E0B1E0E8E0F1E080814A
:1051B00084608C93A8E0B1E0E8E0F1E08081886051
:1051C0008C93A8E0B1E0E8E0F1E0808180618C930D
:1051D000A8E0B1E0E8E0F1E0808180628C93A8E093
:1051E000B1E0E8E0F1E0808180648C93A8E0B1E078
:1051F000E8E0F1E0808180688C9380E293E00E9497
:10520000CF0D88EF96E00E94E71180E092E09F9337
:105210008F9381E08F930E9497140F900F900F90BF
:1052200080E197E00E94E7118DEF91E09F938F93CB
:1052300081E08F930E9497140F900F900F9088E257
:1052400097E00E94E7118AEF91E09F938F9381E0AE
:105250008F930E9497140F900F900F9080E497E027
:105260000E94E71187EF91E09F938F9381E08F93E6
:105270000E9497140F900F900F90A2E0B1E0E2E02F
:10528000F1E080818F7B8C93A2E0B1E0E2E0F1E07D
:1052900080818F7D8C93A2E0B1E0E2E0F1E080813B
:1052A0008F7E8C93A2E0B1E0E2E0F1E08081877F25
:1052B0008C93A2E0B1E0E2E0F1E080818B7F8C93FF
:1052C000AEE2B0E0EEE2F0E090818FE789238C93CC
:1052D000AEE2B0E0EEE2F0E080818F7B8C93AEE254
:1052E000B0E0EEE2F0E080818F7D8C93AEE2B0E042
:1052F000EEE2F0E080818F7E8C93AEE2B0E0EEE2F1
:10530000F0E08081877F8C93AEE2B0E0EEE2F0E0E7
:1053100080818B7F8C93A8E2B0E0E8E2F0E08081AE
:105320008E7F8C93A8E2B0E0E8E2F0E080818D7F90
:105330008C93A8E2B0E0E8E2F0E080818B7F8C9370
:10534000A8E2B0E0E8E2F0E08081877F8C93A8E2F9
:10535000B0E0E8E2F0E080818F7E8C93A8E2B0E0DC
:10536000E8E2F0E080818F7D8C93A8E2B0E0E8E293
:10537000F0E080818F7B8C93A8E2B0E0E8E2F0E07F
:1053800090818FE789238C93A5E0B1E0E5E0F1E01F
:1053900080818F7B8C93A2E2B0E0E2E2F0E090812A
:1053A0008FE789238C93A2E2B0E0E2E2F0E0808113
:1053B0008F7B8C93A2E2B0E0E2E2F0E080818F7D0F
:1053C0008C93A2E2B0E0E2E2F0E080818F7E8C93E9
:1053D000A2E2B0E0E2E2F0E08081877F8C93A2E27B
:1053E000B0E0E2E2F0E080818B7F8C93A2E2B0E05B
:1053F000E2E2F0E080818D7F8C93A2E2B0E0E2E215
:10540000F0E080818E7F8C93A1E3B0E0E1E3F0E0F7
:1054100080818E7F8C93A1E3B0E0E1E3F0E08081B6
:105420008D7F8C93A1E3B0E0E1E3F0E080818B7F9E
:105430008C93A1E3B0E0E1E3F0E08081877F8C937F
:10544000A1E3B0E0E1E3F0E080818F7E8C93A1E303
:10545000B0E0E1E3F0E080818F7D8C93A1E3B0E0E8
:10546000E1E3F0E080818F7B8C93A1E3B0E0E1E3A6
:10547000F0E090818FE789238C93A8E0B1E0E8E029
:10548000F1E080818E7F8C93A8E0B1E0E8E0F1E06C
:1054900080818D7F8C93A8E0B1E0E8E0F1E080812D
:1054A0008B7F8C93A8E0B1E0E8E0F1E08081877F1A
:1054B0008C93A8E0B1E0E8E0F1E080818F7E8C93EE
:1054C000A8E0B1E0E8E0F1E080818F7D8C93A8E076
:1054D000B1E0E8E0F1E080818F7B8C93A8E0B1E05F
:1054E000E8E0F1E090818FE789238C9380E293E0FC
:1054F0000E94CF0D88EF96E00E94E71184EF91E0C3
:105500009F938F9381E08F930E9497140F900F9039
:105510000F9080E197E00E94E71181EF91E09F9367
:105520008F9381E08F930E9497140F900F900F90AC
:1055300088E297E00E94E7118EEE91E09F938F93AF
:1055400081E08F930E9497140F900F900F9080E44A
:1055500097E00E94E7118BEE91E09F938F9381E09B
:105560008F930E9497140F900F900F906CED7FEF28
:1055700080E090E00E94C115DF91CF910895CF9314
:10558000DF93CDB7DEB7A0970FB6F894DEBF0FBE9E
:10559000CDBF0E94FA150E941416009711F00E94C8
:1055A000EC15A8E2B0E0E8E2F0E0808181608C9345
:1055B00068E671E080E090E00E94C115A8E2B0E0EA
:1055C000E8E2F0E080818E7F8C93A8E2B0E0E8E230
:1055D000F0E0808182608C9368E671E080E090E08A
:1055E0000E94C115A8E2B0E0E8E2F0E080818D7F82
:1055F0008C93A8E2B0E0E8E2F0E0808184608C93D4
:1056000068E671E080E090E00E94C115A8E2B0E099
:10561000E8E2F0E080818B7F8C93A8E2B0E0E8E2E2
:10562000F0E0808188608C9368E671E080E090E033
:105630000E94C115A8E2B0E0E8E2F0E08081877F37
:105640008C93A8E2B0E0E8E2F0E0808180618C9386
:1056500068E671E080E090E00E94C115A8E2B0E049
:10566000E8E2F0E080818F7E8C93A8E2B0E0E8E28F
:10567000F0E0808180628C9368E671E080E090E0E9
:105680000E94C115A8E2B0E0E8E2F0E080818F7DE1
:105690008C93A8E2B0E0E8E2F0E0808180648C9333
:1056A00068E671E080E090E00E94C115A8E2B0E0F9
:1056B000E8E2F0E080818F7B8C93A8E2B0E0E8E242
:1056C000F0E0808180688C9368E671E080E090E093
:1056D0000E94C115A8E2B0E0E8E2F0E090818FE717
:1056E00089238C93A5E0B1E0E5E0F1E0808180645E
:1056F0008C9368E671E080E090E00E94C115A5E01F
:10570000B1E0E5E0F1E080818F7B8C93A2E2B0E034
:10571000E2E2F0E0808181608C9368E671E080E0F5
:1057200090E00E94C115A2E2B0E0E2E2F0E08081E8
:105730008E7F8C93A2E2B0E0E2E2F0E080818260B2
:105740008C9368E671E080E090E00E94C115A2E2CF
:10575000B0E0E2E2F0E080818D7F8C93A2E2B0E0E5
:10576000E2E2F0E0808184608C9368E671E080E0A2
:1057700090E00E94C115A2E2B0E0E2E2F0E0808198
:105780008B7F8C93A2E2B0E0E2E2F0E0808188605F
:105790008C9368E671E080E090E00E94C115A2E27F
:1057A000B0E0E2E2F0E08081877F8C93A2E2B0E09B
:1057B000E2E2F0E0808180618C9368E671E080E055
:1057C00090E00E94C115A2E2B0E0E2E2F0E0808148
:1057D0008F7E8C93A2E2B0E0E2E2F0E08081806212
:1057E0008C9368E671E080E090E00E94C115A2E22F
:1057F000B0E0E2E2F0E080818F7D8C93A2E2B0E045
:10580000E2E2F0E0808180648C9368E671E080E001
:1058100090E00E94C115A2E2B0E0E2E2F0E08081F7
:105820008F7B8C93A2E2B0E0E2E2F0E080818068BE
:105830008C9368E671E080E090E00E94C115A2E2DE
:10584000B0E0E2E2F0E090818FE789238C93AEE252
:10585000B0E0EEE2F0E0808184608C9368E671E075
:1058600080E090E00E94C115AEE2B0E0EEE2F0E030
:1058700080818B7F8C93AEE2B0E0EEE2F0E080813D
:1058800088608C9368E671E080E090E00E94C1152A
:10589000AEE2B0E0EEE2F0E08081877F8C93AEE292
:1058A000B0E0EEE2F0E0808180618C9368E671E028
:1058B00080E090E00E94C115AEE2B0E0EEE2F0E0E0
:1058C00080818F7E8C93AEE2B0E0EEE2F0E08081EA
:1058D00080628C9368E671E080E090E00E94C115E0
:1058E000AEE2B0E0EEE2F0E080818F7D8C93AEE23C
:1058F000B0E0EEE2F0E0808180648C9368E671E0D5
:1059000080E090E00E94C115AEE2B0E0EEE2F0E08F
:1059100080818F7B8C93AEE2B0E0EEE2F0E080819C
:1059200080688C9368E671E080E090E00E94C11589
:10593000AEE2B0E0EEE2F0E090818FE789238C9355
:10594000A2E0B1E0E2E0F1E0808184608C9368E65F
:1059500071E080E090E00E94C115A2E0B1E0E2E0D9
:10596000F1E080818B7F8C93A2E0B1E0E2E0F1E096
:10597000808188608C9368E671E080E090E00E940E
:10598000C115A2E0B1E0E2E0F1E08081877F8C9375
:10599000A2E0B1E0E2E0F1E0808180618C9368E612
:1059A00071E080E090E00E94C115A2E0B1E0E2E089
:1059B000F1E080818F7E8C93A2E0B1E0E2E0F1E043
:1059C000808180628C9368E671E080E090E00E94C4
:1059D000C115A2E0B1E0E2E0F1E080818F7D8C931F
:1059E000A2E0B1E0E2E0F1E0808180648C9368E6BF
:1059F00071E080E090E00E94C115A2E0B1E0E2E039
:105A0000F1E080818F7B8C9380E00E948702882F59
:105A100090E098A38F8F81E00E948702882F90E00A
:105A20009E8F8D8F82E00E948702882F90E09C8F4E
:105A30008B8F83E00E948702882F90E09A8F898F56
:105A400084E00E948702882F90E0988F8F8B85E0FA
:105A50000E948702882F90E09E8B8D8B86E00E94AB
:105A60008702882F90E09C8B8B8B87E00E948702B7
:105A7000882F90E09A8B898B88E00E948702882F7C
:105A800090E0988B8F8789E00E948702882F90E0B2
:105A90009E878D878AE00E948702882F90E09C87EE
:105AA0008B878BE00E948702882F90E09A878987F6
:105AB0008CE00E948702882F90E098878F838DE08A
:105AC0000E948702882F90E09E838D838EE00E9443
:105AD0008702882F90E09C838B838FE00E9487024F
:105AE000882F90E09A83898380E197E00E94E711F4
:105AF0002DE332E089899A899F938F938B899C89C2
:105B00009F938F938D899E899F938F938F89988D73
:105B10009F938F93898D9A8D9F938F938B8D9C8D5F
:105B20009F938F938D8D9E8D9F938F938F8D98A133
:105B30009F938F933F932F9381E08F930E949714AD
:105B40008DB79EB743960FB6F8949EBF0FBE8DBF1C
:105B50002CE032E089819A819F938F938B819C8185
:105B60009F938F938D819E819F938F938F81988533
:105B70009F938F9389859A859F938F938B859C851F
:105B80009F938F938D859E859F938F938F85988903
:105B90009F938F933F932F9381E08F930E9497144D
:105BA0008DB79EB743960FB6F8949EBF0FBE8DBFBC
:105BB00088EF96E00E94E71189E092E09F938F932F
:105BC00081E08F930E9497140F900F900F9088E2BE
:105BD00097E00E94E71186E092E09F938F9381E027
:105BE0008F930E9497140F900F900F9080E497E08E
:105BF0000E94E71183E092E09F938F9381E08F935F
:105C00000E9497140F900F900F906CED7FEF80E043
:105C100090E00E94C115A0960FB6F894DEBF0FBEAB
:105C2000CDBFDF91CF910895CF93DF93CDB7DEB78E
:105C300022970FB6F894DEBF0FBECDBF1A8219822D
:105C40000E94A10440E056E960E070E080E00E941C
:105C5000C90540E052EC61E070E081E00E94C905B6
:105C600040E056E960E070E082E00E94C90540E053
:105C700056E960E070E083E00E94C90588EF96E095
:105C80000E94E7110E94700C0E9484150E946C0112
:105C900085E00E94AE0181E00E94CC010E94FA15CD
:105CA00085E892E09F938F9381E08F930E949714F1
:105CB0000F900F900F901A82198216C060E27EE456
:105CC00080E090E00E94C11583E892E09F938F935B
:105CD00081E08F930E9497140F900F900F9089810D
:105CE0009A8101969A83898389819A81813191056C
:105CF0002CF360E777E180E090E00E94C1150E94FC
:105D0000EC150E94BF2AFDCF5058BB27AA270ED002
:105D1000E5C0D6D030F0DBD020F031F49F3F11F455
:105D20001EF4CBC00EF4E095E7FBC1C0E92FE7D02D
:105D300080F3BA17620773078407950718F071F4A8
:105D40009EF5FFC00EF4E0950B2EBA2FA02D0B018F
:105D5000B90190010C01CA01A0011124FF27591BB0
:105D600099F0593F50F4503E68F11A16F040A22FB6
:105D7000232F342F4427585FF3CF46953795279527
:105D8000A795F0405395C9F77EF41F16BA0B620B26
:105D9000730B840BBAF09150A1F0FF0FBB1F661F6D
:105DA000771F881FC2F70EC0BA0F621F731F841FB0
:105DB00048F4879577956795B795F7959E3F08F0D6
:105DC000B3CF9395880F08F09927EE0F9795879595
:105DD000089504D06894B111B5C0089598D088F0A2
:105DE0009F5790F0B92F9927B751A0F0D1F0660FC7
:105DF000771F881F991F1AF0BA95C9F712C0B130E2
:105E000081F09FD0B1E008959CC0672F782F88273C
:105E1000B85F39F0B93FCCF3869577956795B39520
:105E2000D9F73EF490958095709561957F4F8F4F8F
:105E30009F4F0895E89409C097FB3EF49095809594
:105E4000709561957F4F8F4F9F4F9923A9F0F92F40
:105E500096E9BB279395F695879577956795B795BE
:105E6000F111F8CFFAF4BB0F11F460FF1BC06F5FA4
:105E70007F4F8F4F9F4F16C0882311F096E911C0B6
:105E8000772321F09EE8872F762F05C0662371F0D7
:105E900096E8862F70E060E02AF09A95660F771FEB
:105EA000881FDAF7880F9695879597F9089597F9DF
:105EB0009F6780E870E060E008959FEF80EC0895B0
:105EC00000240A94161617061806090608950024D9
:105ED0000A9412161306140605060895092E039453
:105EE000000C11F4882352F0BB0F40F4BF2B11F4C7
:105EF00060FF04C06F5F7F4F8F4F9F4F089557FD26
:105F00009058440F551F59F05F3F71F04795880F27
:105F100097FB991F61F09F3F79F0879508951216BE
:105F200013061406551FF2CF4695F1DF08C016166A
:105F300017061806991FF1CF86957105610508941B
:105F40000895E894BB2766277727CB0197F9089532
:105F50000BD0C4CFB5DF28F0BADF18F0952309F0D5
:105F6000A6CFABCF1124EECFCADFA0F3959FD1F31C
:105F7000950F50E0551F629FF001729FBB27F00DF7
:105F8000B11D639FAA27F00DB11DAA1F649F66274C
:105F9000B00DA11D661F829F2227B00DA11D621F9B
:105FA000739FB00DA11D621F839FA00D611D221F55
:105FB000749F3327A00D611D231F849F600D211D39
:105FC000822F762F6A2F11249F5750408AF0E1F0DC
:105FD00088234AF0EE0FFF1FBB1F661F771F881F25
:105FE00091505040A9F79E3F510570F060CFAACF65
:105FF0005F3FECF3983EDCF3869577956795B79510
:10600000F795E7959F5FC1F7FE2B880F911D969539
:10601000879597F90895629FD001739FF001829F41
:10602000E00DF11D649FE00DF11D929FF00D839F27
:10603000F00D749FF00D659FF00D9927729FB00DC4
:10604000E11DF91F639FB00DE11DF91FBD01CF01D7
:1060500011240895AA1BBB1B51E107C0AA1FBB1F37
:10606000A617B70710F0A61BB70B881F991F5A95E4
:10607000A9F780959095BC01CD01089597FB092E55
:1060800007260AD077FD04D0E5DF06D000201AF4F9
:10609000709561957F4F0895F6F7909581959F4F84
:1060A0000895A1E21A2EAA1BBB1BFD010DC0AA1F59
:1060B000BB1FEE1FFF1FA217B307E407F50720F071
:1060C000A21BB30BE40BF50B661F771F881F991FEC
:1060D0001A9469F760957095809590959B01AC0135
:1060E000BD01CF01089597FB092E05260ED057FD5F
:1060F00004D0D7DF0AD0001C38F450954095309575
:1061000021953F4F4F4F5F4F0895F6F7909580953B
:0E611000709561957F4F8F4F9F4F0895FFCF81
:10611E0064006400620061005E005B005700520084
:10612E004D0047004000390032002A0022001A00BC
:10613E00110009000000F7FFEFFFE6FFDEFFD6FFBC
:10614E00CEFFC7FFC0FFB9FFB3FFAEFFA9FFA5FF8C
:10615E00A2FF9FFF9EFF9CFF9CFF9CFF9EFF9FFF49
:10616E00A2FFA5FFA9FFAEFFB3FFB9FFC0FFC7FF98
:10617E00CEFFD6FFDEFFE6FFEFFFF7FF00000900C0
:10618E0011001A0022002A00320039004000470098
:10619E004D00520057005B005E006100620064001B
:1061AE006400580200005802000058020000580215
:1061BE000000580200005802000058020000580269
:1061CE00000058020000580200005802000028008B
:0261DE0020009F
:00000001FF
